:10000000980B0020E1000000C1000000C1000000CA
:1000100000000000000000000000000000000000E0
:10002000000000000000000000000000C10000000F
:100030000000000000000000C1000000C10000003E
:10004000412D0000FD050000852E000071220000FA
:10005000F1210000252200009D25000065260000FA
:10006000C100000001020000210200004102000066
:100070001D070000D1460000C1000000C1000000C3
:10008000C1000000C1000000C1000000C10000006C
:10009000C1000000C1000000C1000000C10000005C
:1000A000C1000000C1000000C1000000C10000004C
:1000B000A92D0000516C0000C1000000C10000002B
:1000C000064B5921596016215960A0228821596098
:1000D000D205936801210B439360F1E7FC000050C7
:1000E00008B500230C4A0D499A188A4204D20C49DB
:1000F000C95804331160F5E70A4B0B4A191D043B3C
:10010000934203D200221A600B1CF6E704F05AFE59
:1001100000F02EFE08BDC0460000002000010020B7
:1001200044700000040100209807002007B5002358
:10013000019303281ED8114B02301B688000C34076
:10014000181C072318406B46033318701A78002ACE
:1001500002D102F039FE04E01A78022A03D102F03B
:100160006BFE019004E01B78072B05D1044B019333
:10017000019802E0034800E003480EBD140200505D
:10018000008051010197FFFF0297FFFFF8B5071CA0
:100190000E1C012815D9002913D00D1C0124381C70
:1001A000291C06F0B5FD084B821E9A4203D8013C7B
:1001B0002406204307E080230134AD195B009C42F4
:1001C000EDD101204042F8BDFDFFFF00094B402169
:1001D0001A680A431A60084BC022920098580749CF
:1001E00001408020000201439950022200201A6041
:1001F0007047C0460040004000E100E0FF00FFFF04
:1002000008B5054B01219A680A439A60034B1869A7
:10021000DB68984708BDC04620000140000100206F
:1002200008B5054B01219A680A439A60034B586A46
:100230001B6A984708BDC04600001140000100201D
:1002400010B50D4B01219A680C4C0A439A60A36AC1
:100250005B18A362E36A002B0CD0236B002B09D040
:10026000A36B013BA363002B04D1E36B206C984785
:10027000636BA36310BDC046200011400001002045
:10028000034B01225A649A64DA641A657047C046C7
:1002900000010020F0B585B003900C1C151C03284C
:1002A00000D97FE0434B06F01FFD02213F585A6CF6
:1002B000012A79D1586D002876D13F495A658E6858
:1002C00004273E438E603D4E3060B1680A43B26001
:1002D000D86698651C67FFF729FF211CFFF756FFBA
:1002E00003021B0A421C51D1354860E0986C01287A
:1002F0005AD15A6F002A57D12F4958678E6808275C
:100300003E438E602F4E3260B1680143B1601A6087
:100310009A67DC67FFF70AFF211CFFF737FF431CD2
:10032000E2D00302FB4031E0DF6C0197012F3BD1AB
:10033000254A1168002937D11F4E1760B068102771
:100340003843B060214E01983160B7683843B060DF
:100350005160596194600220BDE71F6D0197012F24
:1003600022D11949CA68002A1ED1134ECF60B06845
:1003700020273843B060164E01983260B768384382
:10038000B0609A621A630C610320A4E77360000EE8
:10039000EB0618433060022D08D103980F30C0B22D
:1003A00002F006F80B4802E00B4800E0002005B020
:1003B000F0BDC046000100200002005000000140D6
:1003C0000297FFFF20000140800100200000114043
:1003D000200011400197FFFF0397FFFF73B5002432
:1003E000032800D9BDE0604C06F07EFC02305E8B35
:1003F0006069002800D0B3E00125A5616569013579
:1004000065610190019800282DDC019D142465434D
:1004100056484519AD6D002D15D1019D0126654346
:100420004519AE65019D65434519E965019D654323
:10043000451929660199614341184A66019A544356
:10044000001983668AE001980130DAE7E069002844
:1004500000D085E001252562E5690135E56101905F
:100460000198002801DD00247BE0019D14246543F0
:100470003E482D58002D14D1019D012665432E5074
:10048000019D654345196960019D65434519A96052
:10049000019961434118CA60019A544300190361EC
:1004A0005CE001980130DAE7606A002858D1012544
:1004B000A562656A01356562019001980028D2DC69
:1004C000019D14246543294845196D69002D15D1F6
:1004D000019D0126654345196E61019D65434519DE
:1004E000A961019D65434519E9610199614341187D
:1004F0000A62019A5443001943622FE001980130C7
:10050000DAE7E56A002D2BD118480126C662E66AB3
:100510000136E662019502E0019C01340194019CE0
:10052000002CA0DC019D1424654345192D6B002D82
:10053000F2D1019D0126654345192E63019D654356
:1005400045196963019D65434519A9630199614393
:100550004118CA63019A544300190364019C00E0E6
:10056000034C201C76BDC046800100200001002005
:100570000497FFFF30B503281FD8114B8200D358D2
:10058000104A08309B181968802292050A431A60A5
:10059000C0B20D4BC2220321920001409C58C900F9
:1005A000FF258D40AC4380258D40291C2143995067
:1005B000012282401A60002000E0044830BDC0469D
:1005C000FC6F00000000014000E100E00197FFFF28
:1005D00003280BD8064B8000C358064A00209B18FE
:1005E00019688022D2050A431A6000E00248704769
:1005F000FC6F0000000001400197FFFF084B07B5AA
:100600001A6808219206D20F01921A680A431A60EA
:10061000044B1B6B002B01D00198984707BDC046C7
:1006200000400040800100200C4B01225B68134217
:1006300012D00B4B99680A439A600A4B80211A68C2
:100640008A431A60072210400202074918680840CE
:1006500010431860002000E004487047FC00005080
:100660000002005000400040FFF8FFFF0697FFFF28
:10067000034B40211A680A431A60024B1863704703
:10068000004000408001002008B509283CD806F051
:100690002BFB05090D10191E22262A311B4B802128
:1006A0001A6812E0194B80211A681FE0FFF78EFDCF
:1006B0002BE0164B40211A688A431A60144B022221
:1006C000DA6715E0114B10211A680A430FE00F4B4F
:1006D00010211A680AE00D4B01211A68F5E70B4B4F
:1006E00002211A68F1E7094B02211A688A431A604D
:1006F00000200AE0054B072211400A02186805494C
:10070000014011431960F3E7034808BD0040004071
:1007100004E100E0FFF8FFFF0597FFFF044B10B571
:100720001868044B1B68002B00D0984710BDC046CA
:100730001C000540B4010020824BF7B50D001842A3
:1007400000D0F3E08A79072A00D9F1E0AB23D34047
:10075000DB0700D4ECE00B79032B00D9EAE04B79FE
:10076000012B00D9E8E0CB79062B00D9E6E0A023E5
:10077000DB057549DA688024002805D1640222432C
:10078000DA60DE68714A04E0A4022243DA60DE68BF
:100790006F4A3240DA608B680F2623438B606D4BC3
:1007A000C4180420A3680343A3600223A2681A4369
:1007B000A260EF79A2683E40F0278640BA433243F8
:1007C000A260AE79D03F0640721E9641E268760183
:1007D000BA433243E260AA79E76813405A1E934154
:1007E0001A0110239F433B00012608271343E360AF
:1007F000AA79E3683240D200BB431343E360E36865
:100800002A79053F3A40BB431343E360E2686B79C2
:1008100082431E40B30016001E43E660236A2A7A14
:10082000FB308343134323620A68474BD20703D547
:100830005869494A02400FE01A6AD20305D4586940
:10084000454A02408020400405E01A68520777D5E7
:10085000C0205A69800402435A618E694B6936058B
:10086000360F9B019B0F0136002B02D102F0ACFA30
:1008700007E0354B5B699B019B0F012B03D102F015
:10088000A7FA310001E03100344806F041FA2F6840
:100890000600390006F03CFA0F2305000340626AA7
:1008A000012B0CD87F01B74209D22D4B050913400B
:1008B0006362626A2B4BAF1E134063622EE080219D
:1008C000802389050A436262626A5B051A43264BEC
:1008D000AF1E62629F4221DD0826636A0B4363629A
:1008E000626A204B13406362731C19002800019355
:1008F00006F094FA02290ED80F23616A1B4A1E40A3
:10090000114033060E001E4366620199280006F06E
:10091000FFF9871E02E0019E102EE5D1656AB8B28C
:100920002D0C2D040543656200200AE0104808E004
:10093000104806E0104804E0104802E0104800E0CB
:100940001048FEBDFFFFEFFF00020050FFFFFEFF5B
:10095000FFFFFDFF00000540FFFFFFFC008051018D
:10096000FFFFFFDFFFFFFFEFFFFF0000FFFFFFF0D4
:100970000298FFFF0398FFFF0498FFFF0598FFFF11
:100980000698FFFF0898FFFFF7B501240E002E4BD5
:100990000192C3185D682640A54335434E080227DF
:1009A0002640A6405D605D68BD4335438E08264005
:1009B000BE405D605D68FF19BD4335435D605D68A5
:1009C000CE0826400437F600BD4335435D605E68BF
:1009D0000D09B44662461D4E2540EF0216403E43C7
:1009E00010275E605E682D01BE4335434E098909BC
:1009F00026400C40A10140245D605D68FF1976012E
:100A0000BD4335435D605D68A5432C000C43C321A5
:100A10005C6089000E4B00280BD1019A0D480260E2
:100A2000FF205A5882437F3802435A508022520195
:100A300008E05858084A02408020000202435A50F9
:100A4000802292011A60F7BD00000540FFF7FFFF0A
:100A500000E100E0B4010020FF00FFFF0322F0B539
:100A6000214B224EC018036B214F134303634C7874
:100A70000123621E9441C56A1E4AE4032A402243B0
:100A8000C262C56A8A7814062A02120A2243C26226
:100A90000C78C26A1C40324024022243C2620C78A5
:100AA000C26ADC40144D1C4064022A402243C262E8
:100AB0000C78C26AA4081C40A4023A402243C262D5
:100AC000076ACC780D4A24023A40224302620A792E
:100AD000816813401A020B0033401343836003699B
:100AE0001D400561F0BDC04600000540FFFEFFFF50
:100AF000FFFBFFFFFF7FFFFFFFFDFFFFFF00FFFF8B
:100B000030B5124B0F22DC681025944301221443A8
:100B1000DC60DC68AC43DC60DC6820252C43DC60F6
:100B20005860996019690A431A61BFF36F8F186999
:100B30000121064A0840FAD113689B090B4204D0F0
:100B4000136840210B430248136030BD00C00050C1
:100B50008188FFFF10B5144B0F24DA68A243DA60D6
:100B6000DA681024A243DA60DA682024A243DA604B
:100B7000002258609A601A69012002431A61BFF38B
:100B80006F8F18690124084A2040FAD113689B0925
:100B9000234205D0136840210B431360034801E052
:100BA00092680A6010BDC04600C000508188FFFFF7
:100BB000124B0F21DA688A4302210A43DA60DA68AD
:100BC00010218A43DA60DA6820210A43DA6058602B
:100BD0001A6901210A431A61BFF36F8F1869012155
:100BE000064A0840FAD113689B090B4204D01368E7
:100BF00040210B43024813607047C04600C00050BC
:100C00008188FFFF054B04215A680A435A60044B50
:100C100001211A680A431A607047C046000200505A
:100C200000C00050024B01211A688A431A607047C5
:100C300000C0005010B5162059248821034B5C6079
:100C4000586059605A68002AF9D010BDFC00005065
:100C5000F0B50C0085B0FF2813D102213D4A9368FE
:100C60000B439360FFF7E6FFFFF7CCFFF82040024D
:100C7000FFF79EFFA0220121D20593680B439360EA
:100C8000FEE70130C5B2FF20152D60D8012D0ED131
:100C9000092905D90B1C182900D91823DCB200E05A
:100CA0000A242D4B1B190A3B1A782C4B1A602C4B2B
:100CB000585D0193C0B2844249D0FFF7BBFF802248
:100CC000284B9201DA67FFF79DFFF823DB01EE184E
:100CD000B60003A93000FFF73DFF039B1027234018
:100CE0009C4209D1204B3000E1180391FFF708FF27
:100CF0001EE0013F002F1BD0F8204002FFF758FFF5
:100D0000F82003A94002FFF725FF039B0133F0D130
:100D1000019B5C550024019B195D134BC918F823F6
:100D2000DB01E01880000134FFF7EAFE152CF2D158
:100D300003A93000FFF70EFF039BDCB2FFF772FF41
:100D400080220A4B92011A6001F0E6FF200005B0F4
:100D5000F0BDC046004100500C700000100004407F
:100D6000EB02002004E100E00000FFFF00E100E0F2
:100D7000F0B5594B594F5A4A3B605A4B5A4E1A607C
:100D80005A4A5B4D32605B4A5B4C2A605B4AF9B061
:100D900022608022B2600022BA609A600A23AB60AF
:100DA0002E33A360FFF746FF0121554B1A680A4313
:100DB0001A6008971F00039605950794FB68504A30
:100DC000DB07FBD5116A4F4B4F4C0B4013620C23D2
:100DD00001212360BC3322681A430A4204D12268ED
:100DE0005B0852082260F6E7C02122680902023A35
:100DF0005202386A0A43023B1343DA05400A4002B2
:100E0000D20D02433A62F8229201386A13403F4AF7
:100E1000024013433B623B6A194339623A6A3C4BD6
:100E200013403B623B6A3B4A13403B620E92FB68B5
:100E3000334A5B07FBD5072113698B4305390B4305
:100E40001361D3681B0603D5D3687E310B43D3608F
:100E500003F074FF01F0BCFF2060FFF7D3FEF82021
:100E600012A94002FFF776FE2B4B129A2B4C9A42A6
:100E700011D10025F823DB01E818800012A9FFF743
:100E800069FE129BDBB263550135152DF2D1F925B0
:100E9000234E6D024CE012A92248FFF75BFEF820BA
:100EA000129B4002DBB223750025FFF781FE142D53
:100EB00003D01D4B0F33EB5C6355615D1B4BC918B1
:100EC000F823DB01E818800001351291FFF718FEC6
:100ED000152DECD1DBE7C046FFCF000000400050ED
:100EE000F0FF00004040005080400050FFF700003D
:100EF000C0400050CF5D000000410050D50F000001
:100F000000020050FFFFF7FFD0020020FFC1FFFFEB
:100F1000FFFFFBFFFFFFFEFFA500FFFFEB0200202E
:100F20004F05002050F001000C7000000000FFFF92
:100F300012A92800FFF70EFEF44B129AE918F44BA1
:100F4000100E5854110C3170B270110AF14A043568
:100F5000717004369542EBD11A78FF2A03D1DF3A3B
:100F60001A7000225A7012A9EB48FFF7F3FDFFF741
:100F700059FE002092210126E84BE94A1870129B85
:100F800009061B021B0A13601368E64D5B18136009
:100F9000E54B83221E70032302210093030005F01A
:100FA000FFFD6A6AE14B13408022920013436B629B
:100FB000DF4B1E6005F086FE059B1B6902959B07B3
:100FC00001D404232371079B1B691B0703D404224C
:100FD000637993436371079B1B69DB0607D408227F
:100FE0006379134363716379043A93436371079B95
:100FF0001B699B0607D40822637993436371637965
:10100000043A1343637163791B0705D54022039BA0
:101010009B681343039A936090220025039BA024AE
:101020009B68E4051343039AC24E9360C24BC34AC4
:101030001D70C34B1D70BA4B1B68DBB21370C14AE5
:1010400013701F2311780B401370BF4ABF4B1168F8
:101050000B4003210B431360BD4ABE4B11680B408C
:10106000C02109010B4380211360E26849020A4351
:10107000E260E2680E9B1A40E260BB680B43042109
:10108000BB60B54B9A680A439A609A6802390A4372
:101090009A609A68EE318A439A60DA68D0398A4356
:1010A000DA60DA681D390A43DA60DA6801318A43A6
:1010B000DA60DA688A43DA601A6AFB318A431A62B4
:1010C0007A69A64B13407B61BB691B051B0F049318
:1010D00001F07AFE80223368920513438022336048
:1010E0003368520513433360049B591C05F010FE0E
:1010F0009B4905F00DFE3268023883B2100C0004E3
:1011000018433060226B974B012113400822236360
:10111000236B280093432363236B934AC026134019
:101120002363236BB60013402363904AFFF72CFC24
:10113000142001F03DF98E498E4B0A220B600323E7
:101140000B71012380204D718B71754BCD711B6824
:1011500040031343DBB20B72FFF7EEFA012310A931
:1011600080204B70052340030B708D70CD700D7186
:10117000FFF774FC80202A0001214003FFF704FCE4
:10118000C3227D4C9200A3587C4906200B4080214D
:10119000C9010B43A350290001F092F8022103205A
:1011A00001F074F80321080001F070F8744B0D2071
:1011B0001D7001F0FDF80E2001F0FAF8059A714B50
:1011C0000121D3610523059A5B42936109332360B2
:1011D000A3596D4A03201340A3512A006B4B01F021
:1011E00089F8C022A35912061B021B0A1343A351FC
:1011F00001F09CFA152001F0DBF8012314AE3370E6
:10120000634B2900159332232800169375701795A8
:1012100001F058FD3100280001F0F6FA0121280004
:1012200001F0FEFC0121280001F098FA4E4B594ACA
:1012300051780F93544B04940693554B0B932B000A
:10124000092906D951780E33182902D853780A3B58
:10125000DBB20024504A0125D25C504B504E1A603C
:10126000504B1C70FFF70CF82022BB684E4913430B
:10127000C022BB603460B36880202B43B3607160D0
:101280003368520594461343042233603368C00523
:1012900003433360BB681343BB60444B1C609A68D4
:1012A0002A439A6062465960196811431960FA210D
:1012B0001A68890002431A6028002A00FEF7EAFF34
:1012C0002800FFF785F92800FFF754F92300384A72
:1012D00029002800FFF782F8C222049B92009B5845
:1012E000264AC2211340C02212021343049A8900E5
:1012F0005350022022002F49FEF7CCFF0220FFF7B7
:1013000039F923002C4A2900022057E0000EFEFF85
:101310004E05002018F20100FC0F1000B002002062
:10132000B802002000000E4016030020FFFCFFFF63
:101330001C000050240005409407002044050020B4
:10134000B40200203D0400203C000050FCFCFFFFE4
:1013500030000050F3F3FFFF00000540FFFFFFFCEB
:1013600090D00300FFF7FFFFFFFBFFFF1D460000CB
:10137000D402002020A1070000E100E0FF00FFFFF1
:101380007205002004000400FFFF00FFB5320000DA
:1013900030750000EB0200200C70000010000440CB
:1013A0002000114076050020FFFF000000000140F2
:1013B0009D330000B0360000C9390000FFF70EF879
:1013C000C222049B92009B58C54AC2211340C022EE
:1013D00012041343049A890053502000290001F09D
:1013E000BFFC03227B69062013437B61FFF71CF9D6
:1013F000BC48FFF73DF921000220FFF745F9210025
:101400002000FFF741F901F087FCB74B09961C70EB
:10141000B64B1C80B64B1B78A34204D08023B54A40
:101420001370B54B1D70002301270A930C9304938E
:1014300080330693FFF7FEFBB04A13683B4313600B
:1014400001F06AFCAB4B1B785BB2002B03DBFA228A
:10145000AB4B52001A60AB4B1B685B0728D5FFF7FC
:10146000E9FBFFF7CFFBF920F9244002FFF7A0FBCF
:10147000A54D6402A54BA64AE318D15C2B7809065A
:101480001B04C9186B7820001B02C918AB78043400
:10149000C918FFF735FB9F4B04359C42EAD1FFF793
:1014A000C1FB01F039FC0421964A13688B43136099
:1014B000994B1A68920541D51968984A0A401A60F2
:1014C0008C4A9749127852B2002A01DA052200E0CC
:1014D00000220A700021934A934C11801B682178E6
:1014E000C9B29B0211D408250A20FFF7B1FB23786B
:1014F0008E4CDBB28E4EE37231780B202943FFF71E
:10150000A7FB33781D43257313E008260C20FFF753
:101510009FFB2378854D864CDBB26B7323780D20BF
:10152000BB43237021783143FFF792FB23781E439E
:10153000AE73794A7F4B11680B4013607E4B1B786A
:10154000032B00D022E27D4B1A787D4B1B789A4208
:1015500058D1802370499B040C681C4054D1694BBE
:101560001A68520350D51A683A424DD01A68BA43E5
:101570001A60744B1B78002B46D0802206250B681E
:10158000D20413430B60704B1878C0B2421CD2B225
:101590001A706E4A15541878C0B2451CEDB21D7011
:1015A000052515541878C0B2451CEDB21D701454B1
:1015B0001878C0B2441CE4B21C70654CA446664660
:1015C0002478E4B2651CEDB2357014541878C0B2BA
:1015D000441CE4B21C70862414541878C0B2441C15
:1015E000E4B21C70042414541878C0B2441CE4B251
:1015F0001C70544B1B78DBB213540A68554B1340D4
:101600000B6001E003F02CFC3E4B1B685B0300D435
:1016100035E18020404BC0041968014000D02EE124
:101620001A6802431A601A68120200D4E8E01868C7
:10163000494A02401A602F4B1B785BB2002B00DB3B
:101640008EE020220A24039B414E9B689343039A19
:1016500093603D4B1878C0B2421CD2B21A703B4A1C
:1016600014541878C0B2441CE4B21C7009241454F9
:101670001878C0B2441CE4B21C7011541878C0B27F
:10168000441CE4B21C703478E4B2651CEDB23570D1
:10169000145418783025C0B2441CE4B21C70B22433
:1016A00014541878C0B2441CE4B21C701754187853
:1016B000C0B2441CE4B21C706C4664192478145403
:1016C0001878C0B2441CE4B21C7011541978C9B225
:1016D000481CC0B2187021480078C0B2505480E055
:1016E000FFFF00FF314D000026030020740500209D
:1016F000160300207605002066050020004000400B
:10170000E0020020800700204F050020000EFEFFB1
:101710004E05002018F201006C050020FFFDFFFFC0
:10172000B0020020B202002027030020EB020020BC
:101730007C070020FFFFCFAF940700209507002013
:101740008807002084070020EA0200203F040020D0
:1017500040050020FFFFFFFBFFFF7FFF1503002078
:101760000A24BE4BBE4E1878C0B2421CD2B21A70C8
:10177000BC4A14541878C0B2441CE4B21C7009244A
:1017800014541878C0B2441CE4B21C701154187878
:10179000C0B2441CE4B21C703478E4B2651CEDB2F3
:1017A000357014541878C0B2441CE4B21C70B224D2
:1017B00014541878C0B2441CE4B21C701754187842
:1017C000C0B2441CE4B21C7011541878C0B2441C5E
:1017D000E4B21C7011541878C0B2441CE4B21C70FE
:1017E00011541978C9B2481CC0B218700220505464
:1017F0001978C9B2481CC0B218706B461B7C535490
:10180000994B9A491A68520135D505241A68944EA5
:101810000A401A60914B1878C0B2421CD2B21A70BA
:10182000904A14541878C0B2441CE4B21C700424CA
:1018300014541878C0B2441CE4B21C700024145430
:101840001878C0B2441CE4B21C703478E4B2651C51
:10185000EDB2357014541878C0B2441CE4B21C7058
:10186000B02414541878C0B2441CE4B21C70804BED
:101870001B78DBB213547F4B1A68114019607C4807
:10188000069A03789A4200D1BFE00378764A5BB2A9
:10189000002B47DB0378DBB2069313685B0300D4AD
:1018A000B3E0802205257349D2040B6813430B6013
:1018B0006A4B1C78E4B2621CD2B21A70694A1555A0
:1018C0001C78E4B2651CEDB21D70042515551C781A
:1018D000E4B2651CEDB21D70002515551C78E4B20C
:1018E000651CEDB21D705E4D0D94AC4664462D78BE
:1018F000EDB26E1CF6B226700D9C15551C78E4B244
:10190000651CEDB21D70B02515551C78E4B2651C40
:10191000EDB21D700378DBB213550A68534B1340C8
:101920000B6072E02021039B40249B688B4303994A
:101930008B608021099BC9041B680B4309990B60CC
:101940008021099BC9051B680B4309990B60802105
:10195000089B9B680B4308998B60059B05999B68C6
:10196000A3438B60444BD978444B49001980FA213A
:101970001368490023431360414B196000231C0086
:1019800018A95C520233802BFAD183E7384A0699B2
:101990001378994239D013785BB2002B32DA394B85
:1019A0001B88002B31D12021039B9B688B4303991B
:1019B0008B600421059B34481B690B40FAD18024BD
:1019C000089989682143089CA16040248168A1434B
:1019D00081600220079989688143079881602649C0
:1019E0002648C978490001801F48016821430160E9
:1019F00019001278D2B2069218AA99520233802B9B
:101A0000FAD102E01378DBB20693204B1A88002A41
:101A100000D18EE200221A80029A1D4B126BD2076F
:101A200000D486E21A6B104C3A431A632168194AB3
:101A3000C90331D41968890304D5117818684B009B
:101A400018A9C852029B5B689B0329D510491378DB
:101A500049685B0058A8C15222E0C046EA02002053
:101A6000400500203F04002080070020FFFFFFFB0F
:101A7000760500206C050020EB020020A402002067
:101A8000E0020020E4020020C04000504205002097
:101A900000000E402603002023680E990B402360AF
:101AA000029BDB699B0309D5137838A8DBB2591C6C
:101AB000C9B21170D0495B00C969C1523F23117886
:101AC0000B401370FA22029B12011B689BB29342D7
:101AD00000D8DCE0C94B1B785BB2002B00DBD6E002
:101AE000202240202368C649134323608A78C54BCF
:101AF0001A80226802420BD0226882432260CA7890
:101B0000198852008A1892B21A800022BE4B1A809D
:101B100080214020BD4A93688B439360BC4B9968F9
:101B2000014399603C381D69B9490542FBD18025C4
:101B300090682843906040208A6882438A60B54A52
:101B40001288002AFBD000210720B24A1180B24936
:101B50000A68824380203A430A60029A0001126AAE
:101B60000243029802620298A34A006BC007FAD5AA
:101B70000025106B38431063A84805701068A84D05
:101B800080B2A84204D99F4A1288002AC0D12BE013
:101B900007260868B043802638430860106A36017B
:101BA000304310620298944A006BC007FAD5106B5C
:101BB00038431063106880B2A842E4D8072608684A
:101BC000B043384308608020116A0001014311626C
:101BD000106B8949C007FBD50A6B3A430A630A6850
:101BE00092B2AA42CFD852E0FA21029A09011268B1
:101BF00092B28A424BD98021844A80209268C003E5
:101C00008A438249874D8A6040219A680A439A60D4
:101C1000854A3D391170794A1770844A1168014329
:101C20008348116001780131C9B2017081490D808A
:101C300006787349804D052E0AD98E7A002E01D080
:101C4000897A00E0497AC9B229700021017002E066
:101C5000497AC9B22970002078490880106878490B
:101C600001401160774A1188002910D1202076495F
:101C7000118076498A6802438A602268520306D539
:101C800010219A680A439A601422714B1A6020222C
:101C9000072123689343604A236013688B433B43C7
:101CA00013608022029B12011B6A1343029A136283
:101CB00000231A00180018A9595A0D1C914200D28D
:101CC000151CAAB29508A94201D2801800E040185C
:101CD0000233802BEFD13E2105F01AF8484DC3B2F4
:101CE0000A932B7D984201D2287DC0B22B7D6421BE
:101CF000C01AAF235B00584305F00AF8554B1A6829
:101D0000801840081860FA232A799B005343434AFD
:101D1000984201D20023137023685B0601D500238B
:101D200013708023394E31690B4000D11370A978AC
:101D30001378994249D200231370802240218020D9
:101D4000B368C0039343B360314B9A680A439A6007
:101D5000354A3D391170294A1770344A11680143D8
:101D60001160334908780130C0B208702D488446AC
:101D70006346304803800B782F48052B05D9002394
:101D8000AD7AEDB205700B7002E0697AC9B20170EC
:101D900000202A4908801068294901401160294A19
:101DA0001188002911D120202749118027498A68EC
:101DB00002438A602268530307D51021144B9A68A6
:101DC0000A439A601422224B1A60224B224A1B6853
:101DD0000F2B49D9CF2B02D89B080C3344E01F4965
:101DE0008B4202D81B0933333EE01D498B4239D860
:101DF0009B096C3338E0C04600000E407605002099
:101E0000EB02002092070020A402002000400050B6
:101E1000C04000504205002030000E404D0500201B
:101E20009F0F000088130000B00200206C05002006
:101E30004C050020240300206A050020B202002087
:101E4000FFFFFFBFBE020020DC0500008040005005
:101E500048050020B801002015030020FF04000001
:101E6000FF1400001B0A553B00242000DBB2137056
:101E700038ABE35A0234C018802CF9D1CE4B80091C
:101E80005843CE4B000B98422AD864235B425843F8
:101E9000CB4BAF21C01804F03BFFC3B20493502BCF
:101EA00020D9B368C748A343B360C74B403C9A6886
:101EB00022439A600222027099682143802499602B
:101EC000C24BE400196821431960C1490A7000211E
:101ED0000270C04A11801968BF4A0A401A6016E0B1
:101EE00000230493B94B1A68520510D5049A402A6E
:101EF0000DD81A680F990A401A600022B44B1A7064
:101F0000B64B1978AF4B032900D106321A70002264
:101F1000130058A811007E31415A023A5B18110093
:101F20007E31F7D1FA229B09520053431B0BDBB2DF
:101F30000C93A64803683B4201D1FFF77BFA0F21BF
:101F4000A74B1A788A43C02A0ED19A78D2B25A7017
:101F5000DA78D2B29A701A79D2B2DA705A79D2B2E9
:101F60001A719A79D2B25A710F215A788A43E02AAB
:101F700000D01AE15978D43A0A400C2A00D014E172
:101F80008025924A5C7899781668ED05E4B2C9B26A
:101F90002E4200D1F6E0DB783E2B09D00521894B9B
:101FA000197000218B4B198011688B4B0B4013600B
:101FB0008B4AD378DBB2382B00D1A3E037D82C2B57
:101FC00014D82A2B78D2182B07D80A2B67D2082BC3
:101FD00000D0EAE03E21FF206BE0223B062B00D937
:101FE000E3E0D17808201E39C9B262E0352B6FD00A
:101FF0000DD8332B63D0342B00D0D6E0794C04209D
:102000006179B943FEF724FE6379BB4372E0362B56
:1020100072D0372B00D0C8E008260425714C04206C
:1020200061793143FEF714FE6179A9435AE06D2BC3
:102030001BD8642B37D2492B71D0644A0CD8472B5C
:1020400064D0482B00D0B0E01168674B654C0B4062
:102050001360617920257CE04B2B73D062D34C2B2D
:1020600000D0A2E0036880227AE0812B09D8782B87
:1020700000D380E01423D17802206D395943C9B2CE
:1020800017E0FF2B00D090E00A991320FEF7E0FD47
:102090006A4628215218534B12781A7585E0D17878
:1020A0000020C9B205E00A230920D17864395943D8
:1020B000C9B2FEF7CDFD78E0D17828395FE0494C10
:1020C000042061793943FEF7C3FD63793B4311E096
:1020D00004250826434C280061792943FEF7B8FD02
:1020E0006179B1432800FEF7B3FD63791D43657143
:1020F0006379B343637158E004253A4C2800617951
:10210000A94328E0374C0825617922E08021136833
:1021100049030B43334C1360617920250AE00368BF
:1021200081221DE080211025136849040B432D4CAA
:102130001360617929430420FEF78AFD63791D430A
:10214000657132E010251168284B264C0B40136056
:1021500061790420A943FEF77BFD6379AB43C9E7AE
:102160005205134309220360164B1A706A46194B35
:10217000928D1A8019E02823D17877395943C9B252
:10218000032096E70320044024026418062C0CD197
:10219000DB783E2B09D169460E4B898D1980136877
:1021A0001D4315600822074B1A70084A1368BB4389
:1021B0001360FFF73FF9C04688130000DE020000FD
:1021C000B81E0100B0020020C04000506C05002085
:1021D00076050020B2020020FFFFFFBF9407002019
:1021E00001030020EB020020FFFFEFFFFFFFFFFED7
:1021F00007B5094A136A0093084B196A01910099BF
:102200001162019A1A62064B1B68002B02D00098DB
:102210000199984707BDC04600400050404000501B
:10222000DC0100201FB50E490E4A0B6A0C240193F5
:10223000136A02930C4B186A03900298A043029011
:102240000198086202991162039A1A62074B5B684F
:10225000002B03D001980299039A98471FBDC046EE
:1022600080400050C040005000410050DC01002080
:1022700008B5044B08221A62034B9B68002B00D060
:10228000984708BDC0400050DC0100200A4B800187
:1022900082B0C0180190019B019A01201268884009
:1022A000011C11431960054B20211A6800200A43C4
:1022B0001A6002B07047C046144000508041005080
:1022C00010B50F2810D8094B0F221C6810409443FA
:1022D00020430122186011400A011968102081432F
:1022E00011431960002000E0014810BD80410050FA
:1022F0000189FFFFF7B5294C019400290AD1019902
:10230000019C01262568041C1034A640341C2C4373
:102310000C6014E0012904D1019C019D81402D68CD
:102320000BE002290BD1019C0199061C0D680121CB
:102330000F1C1036B74081403943294321601849AA
:1023400001910121002A06D1019A019C8140246853
:102350008C43211C04E0019A019C814024682143A4
:102360001160C0210F4C104A8900022809D1505831
:10237000E3600E4B034080200004034353500423CA
:1023800008E05058A36000028023000A1B060343A4
:102390005350082300201360FEBDC046DC400050AF
:1023A000D8400050DC01002000E100E0FFFF00FF0A
:1023B00030B5031E1D2B00D9CAE004F095FC0F1B9D
:1023C00022292B323232323232323240464C52588B
:1023D0005F6573828282829090A59EC05D4B0020D3
:1023E00018605D4B18605D4B18605D4B18605D4B6D
:1023F0001860AEE05A4B5C4A19680A408021C90156
:10240000A2E0574B594A19680A40C02189019BE054
:10241000514B00E04F4B1968554A0A40F021090220
:1024200092E04D4A01211068DC1C0D1C053BA540C3
:102430009940A8430B1C011C1943116086E0484BCE
:102440004C4A19680A4004217EE0454B4A4A196803
:102450000A40082178E0424B484A19680A40102196
:1024600072E03F4B464A19680A4020216CE03A4B23
:10247000444A19680A408021490065E0364B424AC7
:1024800019680A4080211AE0354B404A19680A4011
:1024900003210A431A602F4B3D4A19680A40C021A4
:1024A000090151E02C4B3A4A19680A40C021090140
:1024B0000A431A60274B354A19680A40C02189002F
:1024C00042E0264A113B5B000321181C0D1C1468D6
:1024D000994008380B1C85402343AB430BE0214A4D
:1024E0001168192B03D1294B0B40032102E0284B23
:1024F0000B400C210B43136028E0184BFF211A6896
:10250000120C12040A431A60124BFF211A68120CB3
:1025100012040A431A60124B174A19680A408021B4
:1025200009010A431A6019681A4A0A40C0210A437D
:102530001A600C4B0D4A19680A40302104E0094B1F
:10254000144A19680A40C0210A431A60002000E0BA
:10255000114830BD300000503400005038000050A9
:102560003C00005040000050BFBFFFFFCFCFFFFF37
:102570000F0FFFFFFBFBFFFFF7F7FFFFEFEFFFFF83
:10258000DFDFFFFFFEFEFFFFFDFDFFFFFCFCFFFFA7
:10259000F3F3FFFF3F3FFFFF0189FFFFF8B52B4C2F
:1025A000012325681D4205D02360294B1B68002BA1
:1025B00000D0984702231D4205D02360244B9B681E
:1025C000002B00D0984704231D4205D02360204BE8
:1025D0001B69002B00D0984708231D4205D02360BB
:1025E0001B4B9B69002B00D098471A4D1A4C2F6843
:1025F0002668FB0608D52A68184B13402B60144B3D
:102600005B68002B00D09847FB0208D52A68144B62
:1026100013402B600E4BDB68002B00D09847F3066D
:1026200008D522680D4B13402360094B5B69002BD2
:1026300000D09847F30208D52268094B1340236065
:10264000034BDB69002B00D09847F8BD44000440E1
:10265000EC01002050000440540004401F000F0013
:102660000F001F00F8B52B4C012325681D4205D033
:102670002360294B1B6A002B00D0984702231D4280
:1026800005D02360244B9B6A002B00D0984704237D
:102690001D4205D02360204B1B6B002B00D09847B8
:1026A00008231D4205D023601B4B9B6B002B00D0E1
:1026B00098471A4D1A4C2F682668FB0608D52A68D9
:1026C000184B13402B60144B5B6A002B00D09847CB
:1026D000FB0208D52A68144B13402B600E4BDB6AB3
:1026E000002B00D09847F30608D522680D4B134005
:1026F0002360094B5B6B002B00D09847F30208D591
:102700002268094B13402360034BDB6B002B00D086
:102710009847F8BD44001440EC01002050001440DC
:10272000540014401F000F000F001F00084BF02240
:10273000196812040A431A60064BC02219689203F2
:102740000A431A601968044A0A401A607047C04672
:10275000080200500C000050FFFFCFFF70B50726A5
:102760000640321FD3B20125032B0AD91E4CF600B6
:102770002268B5400023AA43994200D02B1C134382
:102780000BE01A4CD200236895402A1C1D1C002324
:102790009543994200D0131C2B432360C30622D5D6
:1027A000103807281FD804F09FFA0406080A0C0EF8
:1027B00010160F4B0AE00E4B0EE00E4B06E00D4BD1
:1027C0000AE00D4B02E00C4B06E00C4B19680C4A7A
:1027D0000A40082105E0094B19680A4A0A4080218D
:1027E00009030A431A6070BD080004400800144041
:1027F0005000044054000440500014405400144061
:1028000007000F000F000700F0B5072385B0039005
:102810001840031C023B0C1C0190B14A052B05D843
:10282000181C04F061FA060608080B0B52699200A6
:1028300006E0526904E0D269920601E0D26912060C
:10284000920F05D0022A06D1A64A1268029204E02D
:10285000A54E029601E0A54F0297039E172E4CD875
:10286000301C04F041FA0C0C0C0C121212124A4AE1
:102870004A4A4A4A4A4A232A2C2E30363B42039F70
:102880009B48F9000568023104E09A48039F0568F7
:10289000F9001E3901228A40E668111C9543002286
:1028A000964200D00A1C2A43026026E0924A9349CD
:1028B0001068E768014039431EE08F4A0AE0904AF9
:1028C0000DE08F4A12E08F4A8C4910680140E068A1
:1028D00011E08C4AE168156808040AE08A4A106829
:1028E0008649E6680140314306E0874AE768156893
:1028F00038048249294001431160019E043EF2B22E
:1029000000962678032A03D97948019F056802E0DA
:102910007848009F0568F900033101228A40111CA4
:1029200095430022964200D00A1C61682A43026047
:10293000002967D1E278052B05D8181C04F0D4F9DA
:10294000050507070C0C714B02E0704B05E0704B5E
:102950001968FF20814304E06D4B110218686D4A2D
:1029600002400A431A606078A5686421684304F055
:10297000CFF9009E01380390F2B20723A678032A0C
:1029800016D9654A01981768191C009787000098A6
:10299000B94088433340BB40011C019E19430C23BE
:1029A00073435E4F1160DA19691E11605C4814E0D0
:1029B0005C4A181C176833400197009F009EB900BD
:1029C000019F88408B4087431F430C23734317604C
:1029D000554F691EDA195548116003991B18196083
:1029E000A3780126032B01D8514AD65CE1780298DE
:1029F000013104F08DF9311C04F08AF9291C04F02E
:102A000087F9FAE0029804F083F98023071C5B053C
:102A100000209F4200D9F0E0464B9F422FD9390C4D
:102A2000381C8EB204F074F980235B02984201D9FD
:102A30000136B6B280235B009E4221D93E0A390E90
:102A4000301CCDB204F064F980235B02984201D9B6
:102A50000135EDB200230122591C171CC9B29F4059
:102A6000AF4201DC0B1CF6E74D1EAA40D5B2002098
:102A7000102D00D9C1E037028026760001E0022641
:102A80000125311C381C04F043F9291C04F040F9DD
:102A9000071C80B2311C0090029804F039F9291CFF
:102AA00004F036F9009904F033F902900198013EE0
:102AB0000238052805D8FF2304F016F909090B0B85
:102AC0003E3E124AFF2113680E408B433AE00F4A04
:102AD00033E00F4A1E40116899430B1C32E0C04698
:102AE00000020050F8000020001BB70000805101D8
:102AF0000800044008001440500004400F000F007C
:102B0000540004405000144054001440000004409D
:102B100000001440FF00FFFF040004400C000440CC
:102B200010000440040014400C0014401000144035
:102B300030700000FFFF0100314A1E40330231496E
:102B400016680E401E43681E16600F2812D804F047
:102B5000CBF8080A110C1111110E111111111111DC
:102B60001110042506E0002504E0012502E00225FD
:102B700000E00325039E6078F60607D5A36864216C
:102B80005F1E5843BFB204F0C3F806E0009E013F49
:102B900070436421BFB204F045F9019A0138043A48
:102BA000D1B280B20723032915D9174A019E1468B0
:102BB000B1001D402E1C8B40251C8E409D4335438B
:102BC000019E0C237343114915605A181760104A6F
:102BD0009B18186010E00F4994000E681D40A34038
:102BE0009E430C235A43A54035430B4E0D60931969
:102BF0001F600A4FD2191060029805B0F0BDC046A0
:102C000000001440FF00FFFF040004400C000440DB
:102C100010000440040014400C0014401000144044
:102C200010220423002921D010420FD0184203D0D3
:102C3000204B14389A6F03E01F4B07219A6F08400E
:102C400001218140081C1043986731E0012218429D
:102C500005D01A4B0438196882400A4327E0184B04
:102C600082401968101C0843186021E010420ED001
:102C7000184203D00F4B14389A6F03E00E4B072114
:102C80009A6F0840012181408A439A6710E001222F
:102C9000184206D0094B04381968824091430A1C37
:102CA00005E0074B82401968101C0A1C82431A6019
:102CB0007047C04600001440000004407C001440EF
:102CC0007C000440072318400322023800B5104B53
:102CD0001140052804D804F007F808080F0F131353
:102CE00058690C4A0907024003E05A6989079200B3
:102CF00092080A435A6109E00901DA69302002E0CA
:102D0000DA698901C02082430A43DA6100BDC04606
:102D100000020050FFFFFFCF034B002058605B68AC
:102D2000DA0700D501487047FC0000500296FFFF0B
:102D3000A023DB059A6801210A439A6070470000CE
:102D400008B5A023DB059A6910210A439A61034B59
:102D50001B68002B00D0984708BDC0462C020020FD
:102D600010B50123232805D10D4A1940C900536825
:102D7000082006E0222808D1094A19405368890032
:102D8000042083430B43536008E0064A83401468E1
:102D9000002901D01C4300E09C43146010BDC046D4
:102DA000000200500802005008B5054B40211A6887
:102DB0000A431A60034B5B68002B00D0984708BD9C
:102DC000000200502C02002000487047001BB70092
:102DD00030B5154B85B06A4623CB23C21B686C46C1
:102DE0001360124B1A6A191C100301D5104A00E037
:102DF000104A096A0D4BCD0312D4186A196A1D6A6C
:102E0000C005C00D89042D04C90EAD0F023050431A
:102E10000231AD0003F07CFF615903F079FF00E05F
:102E2000002005B030BDC0463470000000020050E4
:102E300000805101001BB70010B50E4C072322691A
:102E40001A420CD022691A40022A02D1FFF7C0FFB1
:102E500008E022691340032B03D1074802E007482A
:102E600000E00748A1690F231940013103F050FF2A
:102E700010BDC0460002005010270000001BB70024
:102E800000805101F7B504218020CE4BCE4ADC688A
:102E900011621968C0040143802019601968C005D7
:102EA000014319600021C94BC948198003689B067A
:102EB00034D4C84B1D781900092D2FD8C64D2E6863
:102EC000B6000FD4C54E3678002E0BD029684905C0
:102ED00024D42968490221D419780131C9B2197062
:102EE0001B7809E0BE4B1B78DBB2002B11D00B78AE
:102EF0000133DBB20B700B780A2B0FD18021B94B59
:102F00001970B94B7B39197093683B318B439360CF
:102F100004E00725B4490D70B2490B700021B34B92
:102F20001980C82C00D8BCE10225AB490E680B0003
:102F30002E4200D18AE10E680E352E4202D00B6877
:102F4000AB4314E00E68AA4DB60600D41CE104267B
:102F50000F6837420DD140200B681E430E600A688F
:102F600082430A60AC4200D99BE10B6803430B60CB
:102F700097E180270968B14319601E68BE431E604F
:102F8000AC4202D8196839431960402519681C6899
:102F9000490829402C40A14200D082E11C68954993
:102FA000240600D4DCE00C78012C00D870E1924CAF
:102FB0003F3D64792C423CD0904C2568002D38D19F
:102FC0008F4C276ABC4666468E4F374004262762E0
:102FD0008D4FFE67276A033EB743802627628B4FDB
:102FE000F6053C68344308263C60894C894F2570BF
:102FF000BC683443BC6094683836264396608026AB
:103000000468760234430460834C2570834C257831
:10301000FF2D0FD165780324A543FC2D0AD1804DE7
:10302000AC683443AC60802504686D012C430460B7
:1030300000E008787B4E0C7835787848E4B2EDB241
:1030400005550024250000960E78B44204D8065D8C
:1030500001347540E4B2F7E7002D00D018E13F26B7
:103060000478B443802C57D11968C9000CD5017875
:103070006D4CC9B2217041786C4CC9B2217080246A
:103080001968A400214319605B494C79E4060FD507
:10309000CD7A0478A5420BD10D7B4478A54207D1A7
:1030A00080251C686D042C4300251C60604C258025
:1030B0004C79A40600D4EBE04D7B0478A54200D007
:1030C000E6E001248D7B4178A143A94200D0DFE0F6
:1030D0004178444E21400CD000213E4A117080229C
:1030E00032701968534A0A401A6005223E490A7034
:1030F000CEE0514FB868050080208543BD60402771
:10310000906838439060317081211A6889050A43BC
:103110001A60354A1470BBE01A68484C484E224386
:103120001A602A00474C257001940C783700A44699
:10313000541CE4B2944505D9855CEDB2B554012523
:103140002200F2E7002D01D00198027000980A7861
:103150000078D2B2C0B2B854F2201A6882431A6022
:1031600030480A7800782D4CD2B2C0B2A05420204A
:103170001A6882431A600A780132D2B20A700A7859
:10318000102A00D984E08CE026490A785200D2B295
:103190000A70AC4203D80A780132D2B20A702A49C6
:1031A0000A780132D2B20A700A78072A05D920209B
:1031B0001A6802431A6000220A7010211A680A4332
:1031C0001A606EE020001140C040005070050020E1
:1031D00080070020720500206C05002016030020E7
:1031E0006605002076050020B0020020740500204E
:1031F000FF0500003E040020EB020020E00200205A
:1032000000000E40FFF7FFFF04E100E00000114066
:10321000BC020020804000503F050020C00200207A
:103220000002005017030020270300207C07002025
:1032300086070020FFFFBFDF0040005001000800AC
:103240000103002034020020790700201549164AA6
:103250008C4219D9117812291AD91968490702D54F
:103260001968294319600420196801431960196815
:10327000890716D51968FB30814319601968F5383C
:1032800001431960002309E013780133DBB207E042
:103290001968064A0A401A600023034A1370044A58
:1032A0001370F7BDFF0500007907002000FFFEFF47
:1032B0003E04002008222F4B2F49F0B51A620A68FD
:1032C0002E4B13402E4A0B6013685B0350D58024AD
:1032D0001068A4022B4B204206D1106820431060D6
:1032E00080201C78204306E01468274820401060A6
:1032F0007F201C7820401870802005250B68C004B2
:1033000003430B60214B224F1C78E4B2601CC0B217
:103310001870204805551C78E4B2651CEDB21D708C
:10332000042505551C78E4B2651CEDB21D7000251E
:1033300005551C78E4B2651CEDB21D703D78EDB208
:103340006E1CF6B23E7005551C78E4B2651CEDB2F9
:103350001D70872505551C78E4B2651CEDB21D7003
:1033600013689B03DB0F03550A680B4B13400B607C
:10337000F0BDC046C04000506C050020FFFFDFFFDD
:1033800080070020B0020020FFFFFDFFEA020020BE
:10339000400500203F040020FFFFFFFBF7B5C84AAF
:1033A000C84C1388019401339BB21380C64A13881A
:1033B00001339BB213802388002B03D02388013B69
:1033C0009BB22380C14A13780133DBB21370C04B28
:1033D0001A68002A02D01A68013A1A60BD4A138896
:1033E000002B06D1BC4BBD481A68BD4ED2010FD48C
:1033F00041E01388013B9BB2138013889BB2002BE2
:10340000F0D11900B74AD15401330A2BFBD1E9E7B7
:10341000B54AB6491278802A03D10A88013292B29D
:1034200000E000220A800988B14A914223D9802510
:10343000B04981278A689024AA438A60AE49403DFA
:103440008A68BF052A438A600021AC4A3C3D15705A
:10345000A54A11701A683A431A600768A84A3A40A8
:10346000A84F0260BA682243BA608027A64ABF010B
:10347000D767D5673170A5490A88002A0BD00A881A
:1034800092B2551EADB20D80012A04D120259D496E
:103490008A68AA438A609E490A88013292B20A80E9
:1034A0009C490A88002A03D00A88013A92B20A800D
:1034B000994D9A4A298800290CD02988013989B266
:1034C0002980974911802988002903D14025016866
:1034D000A94301601188002909D01188013989B2F6
:1034E0001180128892B2002A01D18E490A708E4949
:1034F0000A78D2B2002A0ED0FA278C4DBF006A8813
:10350000BA4202D801326A8014E000226A800A7846
:10351000013AD2B20DE08649097800290AD07249F1
:10352000097849B2002905DB1D68824929401960E4
:1035300081490A70814A118889B24D1CADB215804B
:10354000C8291DD180276B4DA968B943A9606A4D70
:10355000403FA9683943A9600021774D3A3F29705F
:10356000774D29801D687749294019605E49634D70
:103570000F703178C9B2002901D1297000E02F7095
:103580001288C72A21D81A6852041ED50021402764
:10359000694A584D1170AA6880310A43AA60564D95
:1035A000AA68BA43AA60504A1170544A7B39117014
:1035B0001968654A0A4080211A600268C9040A43F2
:1035C00002601968614A0A401A60614A116800295C
:1035D0000AD01168013911601268002A04D110253F
:1035E00045498A68AA438A605A498A79002A0FD0D5
:1035F0004E4A97887D1C95800A258C796543AF4299
:1036000006D180271D683F043D431D60002595803D
:10361000514A15880135ADB215803578EDB2002DCF
:1036200000D1ADE04D4D296801312960C8212F68D6
:1036300089008F4200D8C4E000212960484D2F68DE
:103640000F253D40474F40353D709027464D317026
:103650002970464D2B4E2970B5683D43B560012653
:10366000334D103F2E70234EB568BD43B560224EDA
:10367000403FB5683D43B560204D019C2970304DF9
:1036800029801E682F4D354004261D60384D2E6060
:10369000FA25AD0025800625134C2570264C217097
:1036A0001D68294C25401D60324C02252170324C8A
:1036B000217032498C6834438C608C6878E0C04655
:1036C00028030020E40200207A0700204D05002096
:1036D000E00200203A0300206C0500208007002053
:1036E000940700201803002076050020860700209C
:1036F000B036000000400050C0400050B002002032
:10370000FFFFFBFF8040005004E100E0BE0200200C
:103710004205002092070020A4020020240300207C
:10372000881300004C0500206A05002034020020A8
:1037300016030020FFFFBFFF720500207405002064
:10374000B2020020FFFFFFBFFFFFBFDFFFBFFFFF91
:1037500048050020EB020020680500208C070020AF
:10376000B80200203D0400207807002095070020C3
:1037700000E100E0EA020020880700200000154078
:10378000497949071DD5874C218889B24E1CB6B2AC
:103790002680FA26B600B14213D925801025824929
:1037A0000C692C4206D08C68AC438C608C687035F8
:1037B0002C4305E08C682C4380258C608C68AC43DE
:1037C0008C60802100688902084035D01388DBB204
:1037D000802B00D0E5E0754A754B9179012916D010
:1037E00000290AD002291ED198680143042099605B
:1037F000996881439960032313E004209968014389
:1038000099609968023881439960012309E0022098
:1038100004249968014399609968214399609071E3
:10382000BFE09371BDE0002191719A6802318A4333
:103830009A609A680231B2E05E495F4C0D88002DB3
:1038400013D00D88012D0CD11E685C4D35401D60D4
:103850005B4B1B785BB2002B02DA0523237000E080
:1038600020700B88013B9BB20B802078C0B20928E6
:1038700000D996E003F038FA05132A303D5C6177F1
:103880007B82FA224F4B92001988914200D088E047
:10389000002204211A80464A93684B403FE0138877
:1038A0008022DB05DB0D5200934200D079E03F4BD4
:1038B000D879421CDA71052873D803F015FA03325F
:1038C000033272363A4A0421936827E012880221B3
:1038D000374B92060BD504E012880221344B1206B6
:1038E00005D59A680A439A609A68491857E09A6819
:1038F00055E013888022DB05DB0D5200934250D146
:103900002A4BD879421CDA7105284AD803F0ECF921
:1039100003090309490D0221254A93680B4393606B
:103920003FE0234B04219A6835E00022DA7138E049
:1039300004211F4B9A680A432EE0FA22214B920081
:10394000198891422DD100221A80184B1A7A511CE5
:1039500019720421164BD2071CD49A680A439A6044
:103960009A68022114E0124B04219A680CE0128834
:1039700004210F4B52060DD59A6809E012880421E4
:103980000B4B520606D59A680A439A609A68023928
:103990000A4305E09A688A4302219A609A688A433A
:1039A0009A60F7BD7005002080400050340200206E
:1039B00000410050B2020020B0020020FFFFFFBF14
:1039C00076050020740500208022AA4BF0B5196806
:1039D00052021143A84C1960207885B0C0B2411C36
:1039E000C9B22170042801D900F008FE03F07CF967
:1039F0000C030C0C1400A1498B681A438A6008213F
:103A00009F4A93688B43936080219E4AC90513683F
:103A10000B43136000F0F2FD80209B49C0040A783C
:103A2000013AD2B20A70994A1168014380201160AC
:103A30001168C005014311609549D0688842FCD9DE
:103A400000260120934A04251670934A1670934A63
:103A5000116A0143894811628468914921404024D8
:103A60008160904988688C46A04388608E480560D4
:103A70008025106A2D01284310628C484279224229
:103A800001D100F012FD8A4D2C782A00B44201D1F8
:103A900000F00BFD2C780F2C01D800F006FD2C78DF
:103AA000EF2C01D900F001FD2C78824F0F3CE4B2DD
:103AB0003C5DE7B27F4C402F63D11A68D20401D439
:103AC00000F0F3FC1B685B0301D400F0EEFC8022E5
:103AD0000A247949D2040B68784F13430B60784B62
:103AE0001878C0B2421CD2B21A70764A14541878B0
:103AF000C0B2441CE4B21C70092414541878C0B23B
:103B0000441CE4B21C7016541C78E4B2601CC0B2B1
:103B100018703878C0B2451CEDB23D701055187859
:103B2000C0B2441CE4B21C70B32414541878C0B260
:103B3000441CE4B21C70FF2414541878C0B2441C16
:103B4000E4B21C7016541878C0B2441CE4B21C7065
:103B500016541878C0B2441CE4B21C70165418787D
:103B6000C0B2441CE4B21C7016541878C0B2441C95
:103B7000E4B21C7016540A68534B13400B6000F0FB
:103B800094FCBE0801966E463679072E44D003D8C1
:103B9000002E08D000F089FCBE080E3E012E00D891
:103BA000A3E100F082FC10208A6882438A606A7870
:103BB00040490F3A8A5CD2B20292402A01D100F009
:103BC00074FC424A117849B2002904DA3F21107886
:103BD000084001900AE09178C9B2D1705178C9B219
:103BE00091701178C9B25170002101910F20917824
:103BF00081430020E02901D09070D070002134482A
:103C0000465C555C0400AE4201D000F0EDFC013191
:103C10000529F5D100F076FC10268D68B5438D603E
:103C200091780F2907D9D178EF2904D891780F39E5
:103C3000C9B2615CCFB2012F06D0002F07D0072F89
:103C400000D1C8E000F031FC80256D0000E03D00AF
:103C500011780F39C9B2665C52781C490F3AD2B25A
:103C6000A25CF6B2D7B20A7852B2002A32DA0A78E7
:103C700039E0C04680070020BC020020000200504E
:103C80008040005000001140260300202000114019
:103C900061020000790700203E04002000000E4071
:103CA000FFFFFEFFC040005000E100E0EB020020FB
:103CB000A6020020000000206C0500204005002026
:103CC000EA0200203F040020FFFFFFFBC0020020AB
:103CD000180300208A78D2B2CA704A78D2B28A70A9
:103CE0000A78D2B24A7000240A78019452B2A242F1
:103CF00003DA3F220C78144001941B685B0300D464
:103D0000D3E3ED49B2014B89BA18D2B2D218AA183E
:103D100092B252084A8143795BB2002B00DBC4E3C4
:103D20000A23E6490D88C07C43439D4200DCBCE386
:103D300000260E8080210827E148C90403680B4350
:103D40000360E04B1D78EDB2691CC9B21970DE4901
:103D50004F551D78EDB26F1CFFB21F7007274F55EE
:103D60001D78EDB26F1CFFB21F704E551D78EDB27D
:103D70006E1CF6B21E70D54EB44664463678F6B266
:103D8000771CFFB227704E551D786C46EDB26E1C45
:103D9000F6B21E70A6264E551D782479EDB26E1C23
:103DA000F6B21E70CA4E7678F6B24E551D78EDB258
:103DB0006E1CF6B21E704C551C78E4B2651CEDB258
:103DC0001D70D5B20D551C78120AE4B2651CEDB217
:103DD0001D700A55C0E211780F39C9B2615CC9B2D1
:103DE000019152780F3AD2B2A25CD2B20292B84A92
:103DF000147864B2002C03DA14783F22144009E0EE
:103E00009478E4B2D4705478E4B294701478E4B244
:103E100054700024827C002A00D146E36422AD4D18
:103E20002E88807C4243964200DC3EE300262E80B2
:103E30001B685B0300D438E380220927A048D20422
:103E40000368134303609F4B1D78EDB26A1CD2B226
:103E50001A709D4A57551D78EDB26F1CFFB21F7046
:103E6000082757551D78EDB26F1CFFB21F705655CD
:103E70001D78EDB26E1CF6B21E70944EB4466146CB
:103E80003678F6B2771CFFB20F7056551D78EDB23A
:103E90006E1CF6B21E70AA2656551D78EDB26E1C29
:103EA000F6B21E70FF2656551D78EDB26E1CF6B2A6
:103EB0001E70874E7678F6B256551D78EDB26E1CA0
:103EC000F6B21E7054551C78E4B2651CEDB21D703C
:103ED000012515551C78E4B26519EDB21D70019BE2
:103EE0009901029B5918C9B235E21968C90400D476
:103EF000DBE26146102089688143604681606A7810
:103F0000734D0F3AA45C6878B901FB38C9B2E4B2CA
:103F1000042800D9C9E202F0F1FE240205000500E0
:103F2000E300E30080221B68D202402C00D188E02D
:103F3000134200D1B9E280220A26614BD2041B68E9
:103F4000214313435E4A13605E4B1A78D2B2501C71
:103F5000C0B218705C4886541A78D2B2561CF6B2B9
:103F60001E70092686541A78D2B2561CF6B21E70FC
:103F7000002686541A78D2B2561CF6B21E70534EE2
:103F8000B44665463678F6B2771CFFB22F70865479
:103F90001A78D2B2561CF6B21E70B32686541A781E
:103FA000D2B2561CF6B21E70FF2686541A78D2B2D0
:103FB000561CF6B21E70484E8154B278474C0F3AE8
:103FC000A25CF17892010F39615CD2B20A43197890
:103FD000C9B24F1CFFB21F70425432790F3AA15C34
:103FE000727989000F3AA25CC9B2D2B2170939437B
:103FF000009169461F781201FFB27D1C0D710D7989
:1040000000991D70C155B179D2B20F39615CC9B246
:104010008F083A4300926A461F788901FFB27D1CDF
:1040200015711579009A1D70C255F2790F3AA25C8C
:1040300011431A78C9B2D2B2541CE4B21C70815434
:104040002DE2134200D130E280220A241C48D2041F
:1040500003681E4F134303601A4B1978C9B24A1CF8
:10406000D2B21A70184A54541978C9B24C1CE4B22E
:104070001C70092454541C78E4B2611CC9B2197034
:10408000002111551D78EDB26C1CE4B21C703C7817
:10409000E4B2661CF6B23E7054551C78E4B2651C5E
:1040A000EDB21D70B32515551C78E4B2651CEDB258
:1040B0001D70FF2531E1C046340200202803002096
:1040C0006C050020EA0200203F040020400500208B
:1040D000C00200207A070020A60200200000002075
:1040E00080221B68D202402C00D1B1E0134200D1E3
:1040F000DBE180220F26F84BD2041B6821431343D7
:10410000F54A1360F54B1878C0B2421CD2B21A704F
:10411000F34A16541878C0B2461CF6B21E70042634
:1041200016541878C0B2461CF6B21E7000261654FB
:104130001878C0B2461CF6B21E70EA4EB446654608
:104140003678F6B2771CFFB22F7016541878C0B2CA
:10415000461CF6B21E70B42616541878C0B2461C1F
:10416000F6B21E70FF2616541E78F6B2701CC0B24E
:104170001870DD488778FFB297551E78DB4CF6B291
:10418000771CFFB21F70C778FFB297551E78F6B242
:10419000771CFFB21F700779FFB297551E78F6B2F1
:1041A000771CFFB21F704779FFB297551E78F6B2A1
:1041B000771CFFB21F708079C0B290551878C0B2DA
:1041C000461CF6B21E70CA4E1154B1780F39615CAC
:1041D000F07889010F38205CC9B201431878C0B269
:1041E000471CFFB21F70115431790F39605C71792F
:1041F00080000F39615CC0B2C9B20F09384300902A
:1042000068461F780901FFB27D1C05710579009889
:104210001D70D055B079C9B20F38205CC0B2870884
:104220003943009169461F788001FFB27D1C0D71F2
:104230000D7900991D70D155F1790F39615C0843F2
:104240001978C0B2C9B24C1CE4B21C70505426E1BB
:10425000134200D129E180220F249F48D204036831
:10426000134303609D4B1978C9B24A1CD2B21A702D
:104270009B4A54541978C9B24C1CE4B21C700424F3
:1042800054541C78E4B2611CC9B219700021115554
:104290001C78E4B2661CF6B21E70924E0194B446CD
:1042A00064463678F6B2771CFFB22770019C16552B
:1042B0001C78E4B2661CF6B21E70B42616551C7843
:1042C000E4B2661CF6B21E70FF2616551C78E4B2E6
:1042D000661CF6B21E70AE78F6B216551C78E4B2C3
:1042E000661CF6B21E70EE78F6B216551C78E4B273
:1042F000661CF6B21E702E79F6B216551C78E4B222
:10430000661CF6B21E706E79F6B216551C78E4B2D1
:10431000661CF6B21E70AD79EDB215551C78E4B28C
:10432000651CEDB21D7011551C78E4B2651CEDB230
:104330001D7011551C78E4B2651CEDB21D7011554D
:104340001C78E4B2651CEDB21D7011551C78E4B206
:10435000651CEDB21D7011550268664B1340036079
:10436000A3E0402C00D1A0E01B685B0300D49CE0DC
:1043700080220A26584BD2041B6821431343564A15
:104380001360564B1D78EDB26A1CD2B21A70544AB3
:1043900056551D78EDB26E1CF6B21E7009265655A4
:1043A0001D78EDB26E1CF6B21E70002656551D78B3
:1043B000EDB26E1CF6B21E704A4EB44660463678B8
:1043C000F6B2771CFFB2077056551D78EDB26E1C21
:1043D000F6B21E70B52656551D78EDB26E1CF6B2BB
:1043E0001E70FF2656551D78EDB26E1CF6B21E707B
:1043F0003F4E5155B1783D4D0F39695CF4788901D4
:104400000F3C2C5DC9B221431C78E4B2671CFFB29B
:104410001F70115531790F396C5C7179A4000F3917
:10442000695CE4B2C9B20F093C4300946C461F7842
:104430000901FFB2781C20712079C9B21870009868
:10444000D055B4790F3C2C5DE4B2A70839430091F4
:1044500069461F78A401FFB2781C08710879009999
:104460001870D155F1790F39695C0C431978E4B2B1
:10447000C9B24D1CEDB21D70545419781A4DC9B211
:104480004C1CE4B21C70EC79E4B254541C78E4B2D5
:10449000611CC9B21970C023297A0B4313550E4B06
:1044A0001A68144B13400C4A13601021124B1A68FF
:1044B0000A4205D00320114A10601A688A431A6024
:1044C00019680F4A0A401A6000231900084AD1549B
:1044D0000133082BFBD191E06C050020EA0200209B
:1044E0003F04002040050020C00200200000002002
:1044F000A6020020FFFFFFFB8007002048050020E8
:10450000FFEFFFFF3E49087B844601300873614698
:104510000329CAD11B685B0361D58021092539486D
:10452000C90403680B430360374B1C78E4B2611C79
:10453000C9B2197035490D551C78E4B2651CEDB24D
:104540001D7008250D551C78E4B2651CEDB21D7078
:1045500000250D551C78E4B2651CEDB21D702C4D84
:1045600003942D782A4CEDB26E1CF6B22670039C93
:104570000D551C78E4B2651CEDB21D70A5250D55D6
:104580001C78E4B2651CEDB21D705578EDB20D5586
:104590001C78E4B2651CEDB21D706D462D790D5589
:1045A0001C78E4B2651CEDB21D70D578EDB20D55E6
:1045B0001C78E4B2651CEDB21D70654692782A4005
:1045C0000A551A78D2B2541CE4B21C70BB01029C8A
:1045D000DBB223438B5402680E4B13400360C822A6
:1045E0000D4B92001A8060E7002305490B73D15CE4
:1045F000C9B2E1540133052BF9D156E705B0F0BD3E
:10460000340200206C050020EA0200203F04002054
:1046100040050020FFFFFFFB3A030020F7B56A4684
:10462000234BD01D1B680127DBB2037000231D0044
:104630001E001C0001781F4AC9B251739373D373D3
:10464000082B09D0394202D001260134E4B20133EB
:104650004908DBB20125F3E7002E00D09473002D4A
:1046600002D008235173D373937B042B1FD1124BB9
:104670001A68520307D51024104A916821439160AB
:104680001A6822431A600E490B78DBB25A1CD2B268
:104690000A7002780B48D2B2C2540B78092B06D9A3
:1046A0000023094A0B709168084B0B409360F7BDDB
:1046B000000005403402002080070020C040005068
:1046C0003F050020A602002000020050FFFFFEFF71
:1046D000F0B5BD4C87B0236804AADBB2D11D0B70C6
:1046E000A3691B07DD0F002B00DB51E108264027E3
:1046F0007F22A3693343A36108780B7838401340C5
:10470000002800D1BCE07D2B00D1B5E07E2B00D08D
:10471000BAE2AE4D2B78002B00D08DE08021AC4A60
:1047200093688B439360AB4A93681F43AA4B97608F
:104730001B78DBB2002B06D08021A84AC901136880
:104740000B43136004E00621A54A1170A54A1370BB
:10475000A54A1378DBB2002B03D01378013BDBB200
:1047600068E00B22A14DA2492A70013A6A70E63234
:10477000AB70EB702A71EE3A6A713C32AB71EA7140
:104780000A68120E2A720A68120CD2B26A720A6899
:10479000120AD2B2AA720A680C21D2B2EA72954AFF
:1047A0001170954A1370954A13748C4A944B116892
:1047B0000B4013601022E3681343E360E368921830
:1047C0001343E360E368183A1343E360A369DB0033
:1047D000FCD52E787C4BF6B21E60300000F01CFB3E
:1047E0000127B74215D8A3691B02FCD4824A764937
:1047F000137801370133DBB21370EB5CFFB2DBB22D
:104800000B601378DBB2EB5C5840C0B200F004FBE5
:10481000E7E7A3691B02DB0FFBD16B4A7649106007
:104820000A780132D2B20A70764A1370764A13605F
:10483000664A0233137046E22B78022B00D042E224
:1048400000F0DCFA0021684B6F4A18706F4829703D
:10485000116011684C1C14608142FAD9002111606A
:104860001A788A4200D02EE2614A1268D2B21A70D7
:104870000F2219780A405BE00022634B1A6022E2A3
:10488000002B17D180245F4864000278D2B2511CFB
:10489000C9B201705E49520054520278520053521C
:1048A00080210378554ADBB213745A4A090613680B
:1048B0000B4366E0454B1B78DBB2022B63D0032B26
:1048C00000D0E1E1544B09781A781F230B40934242
:1048D00000D0F8E110214C4A1060E3680B43E3601C
:1048E000E36849180B43E360E3683343E3600292F3
:1048F000A3693549DB00FBD5384B1A688023DB04FC
:104900001A4002D001230B60DDE13B4B39481F7890
:1049100005781E00AF4201D10A60D4E11A78334D08
:10492000D2B2AD5CEDB22A1F3B2A03D90278D2B2D3
:104930001A70C8E10D60280000F06EFA0127A36923
:104940001B02FCD43378294A0133DBB23370D35CC9
:104950001D49DBB20B6033780137DBB2D35CFFB2A9
:104960005840C0B200F058FABD42E8D2A3691B0219
:10497000DB0FFBD1144A106032780132D2B23270B0
:10498000029A13609FE11D4B1D741F4B18607BE161
:10499000204A1C4D10681E4B002800DB5FE1174EBB
:1049A000307C40001F5AC0203840029036D0116839
:1049B0004900490811600021327C013AD2B22A70C4
:1049C0002A78520099527EE1000015409407002099
:1049D00000400050C0400050160300206C0500202D
:1049E000B0020020760500203D0400203F04002096
:1049F000B8020020EA0200209007002034020020C4
:104A0000FFFFFFFB880700208C070020FFFF0F003F
:104A100078050020800700203C0400202F78F8B2A1
:104A2000019002AF0130F871F87928700198097887
:104A30004700D953317C4900595A002900D123E15C
:104A4000317C49005F5A317C2E780231C919C9B2D4
:104A5000B14200D018E1297802A8C9B24E1CF6B2C2
:104A60002E7080264900B6005E52297800884900E1
:104A700058520298136806005B005B081360934F5E
:104A8000934A3B7C39005B009B5A0133B3420FDBF6
:104A90003B7CF318DBB25B009B5A8E4ADBB293552A
:104AA000935D01365840C0B200F0B6F9F6B2E6E7C1
:104AB000894A1378DBB2022B05D0032B00D0E3E048
:104AC0000022864BC9E0834B002804D000231370DA
:104AD000FF22834B2CE71A791E00702A7ED1002119
:104AE0007E4F804E3960587A3268120E904200D064
:104AF000CAE09A7AFF2094463268120C024094452C
:104B000000D0C1E0DA7A94463268120A0240944535
:104B100000D0B9E01A7B36680640B24200D0B3E05C
:104B200003226D4E32705B796F4ADBB213701378DB
:104B3000DBB28B4203D13370694B1870C3E039602C
:104B40002B786A4ADBB21370694B6A4A18680240D4
:104B50001A60694A69485579AD0718D58027684EAB
:104B60000170B568BD43B560664E403FB5683D43D2
:104B7000B560654D297065490D78052D01D1023567
:104B800000E006250D70002561490D7001E001214E
:104B90000170102551799026A943517152790C3D2D
:104BA0005C492A4216D08A68B2438A600278002A99
:104BB0006AD00021584A11801868584A02401A6089
:104BC000574A1560524A1170564A11701968564A70
:104BD0000A4042E08B6833438B6055E01A79722AB1
:104BE0001FD100253D4A3F481560597A0268120ED0
:104BF000914249D1FF219E7A0268120C0A409642E6
:104C000042D1DE7A0268120A0A4096423CD11A7BEF
:104C100003680B409A4237D12F4B1D70304B1970EF
:104C200051E018781F785A78C0B2013297422BDDD4
:104C30005A780132D2B20A740F7C1A78D21BD2B2DF
:104C40001A7000220132D7B2B84200D843E70F7C75
:104C5000BF18F75DFFB2B754F4E71A6014E0287884
:104C6000013840001E5A8020400086420CD128782E
:104C7000C0B2461CF6B22E7009784000195280214D
:104C8000136809060B431360A369284A1B0403D564
:104C9000022193680B439360A269244BD20707D586
:104CA00001219A690A439A619A6849180A439A60ED
:104CB000A3699B0603D41D4B9B69DB0603D5022227
:104CC000A3681343A36007B0F0BDC04634020020C0
:104CD000780500203C030020940700208C0700206A
:104CE0003D040020B80200203C040020950700206D
:104CF0006C050020FFFFFBFFEB02002016030020E5
:104D000000400050C040005066050020B002002066
:104D10007605002080400050B2020020FFFFFFBF58
:104D200000E100E072050020FFFFBFDF000015403A
:104D300010B5FBF77FFFFDF7FBFF10BD70B51B4CF7
:104D4000072322691A4E1340052B02D8022B04D0E8
:104D500000E004239B00F0581AE0256A01232D048B
:104D6000AD0FAB4292415242AD1A226AD20C1A42A6
:104D700001D0104B00E0104B206A216AC005C00D25
:104D80008904C90E02305843023101F0C1FFE840E6
:104D9000A1690F231940013101F0BAFF074B70617F
:104DA0000749C01801F0B4FFB06170BD00020050A7
:104DB000E400002000805101001BB70020A1070083
:104DC00040420F00704700000B4B1A7819785200D0
:104DD000D2B24A4052001978D2B24A401201197830
:104DE000D2B24A401978D20949005218D2B21A7088
:104DF0001878C0B27047C0464405002010B5FFF7D0
:104E0000E3FF0F23034A18401378C0181F231840EC
:104E1000107010BDB40200200023C20700D55E331D
:104E2000820701D5BC225340420701D5612253407D
:104E3000020701D5C2225340C20601D59D2253402C
:104E4000820601D523225340420601D54622534013
:104E500040B2002801DA8C2253401800704700004D
:104E6000F0B5D24BD24C1A78237893B09A4201D144
:104E700001F064FE80232278CE4D5B00002A12D11F
:104E8000FF32FF32AA5A19009A4202D18022520000
:104E900015E02378DBB25A1CD2B222705B00EB5AC9
:104EA0008B42F6D1F2E72278013A5200AA5A9A428E
:104EB000ECD02278D2B2511CC9B22170F5E7237828
:104EC0005B00EB5A934204D123780133DBB22370A9
:104ED000F5E723785B00EB5A002B01D101F02EFEA1
:104EE00023785B00EB5A0233DBB20193019A2378FB
:104EF000D318DBB25B00EA5A80239B009A4201D0B0
:104F000001F01CFE002630002378019AD318DBB292
:104F10005B00EE52019AF3B29A420FD92278D2B2D4
:104F2000531CDBB223705200AA5AD3B202AA935583
:104F30004340D8B2FFF770FF0136EBE780222378B9
:104F40009D490133DBB223700B68D20413430B601D
:104F5000002845D0994B02AA1B7892789A423FD1FB
:104F600000200625964B974F18701C78E4B2621CFF
:104F7000D2B21A70944A15551C78E4B2651CEDB291
:104F80001D70052515551C78E4B2651CEDB21D7029
:104F900010551C78E4B2651CEDB21D703D78EDB281
:104FA0006E1CF6B23E7015551C78E4B2651CEDB26D
:104FB0001D70862515551C78E4B2651CEDB21D7078
:104FC000022515551C78E4B2651CEDB21D7002ABCC
:104FD0001B791355754B18707C4B186001F0D7F98D
:104FE000012702AB9D78754B1A781C00954211D1B0
:104FF000774A02A9107809790130884209D01078DF
:10500000744EC0B23070002903D0734E30683843FC
:10501000306011701B789D4201D001F00AFC8021A4
:10502000654AC90413680B43136002AB5B79110036
:10503000102B01D100F081FD00D999E0072B00D1A0
:10504000FEE14DD8032B00D155E13FD8012B00D113
:105050000EE1022B01D001F0ECFB06200526584B97
:105060001978C9B24A1CD2B21A70574A50541978EA
:10507000C9B2481CC0B2187056541978C9B2481C3D
:10508000C0B21870002050541978C9B2481CC0B280
:1050900018704C48844665460078C0B2441CE4B29F
:1050A0002C7050541978C9B2481CC0B218708320B3
:1050B00050541978C9B2481CC0B2187056541978A7
:1050C000C9B2481CC0B218700023EAE1052B00D118
:1050D00057E100D906E3404A404B11680B404DE1CF
:1050E0000B2B00D1B9E308D8092B01D101F061FBEA
:1050F000334A354900D82EE3DAE30E2B00D174E3AE
:1051000001D901F015FB0C2B01D001F092FB052019
:105110002B4B2C4D1978C9B24A1CD2B21A702A4AAC
:1051200050541978C9B2481CC0B2187004205054A9
:105130001978C9B2481CC0B21870002050541978B0
:10514000C9B2481CC0B218702878C0B2441CE4B27E
:105150002C7050541978C9B2481CC0B218708B20FA
:1051600050541978C9B2481CC0B21870FF2398E196
:10517000172B01D101F09CF932D8132B01D100F08B
:1051800084FF09D8112B01D100F08FFD122B01D122
:1051900000F03EFD01F04DFB152B01D101F03DFA71
:1051A00001D801F06FFA01F0E4F8C046880700204A
:1051B00095070020780500206C0500203C040020A5
:1051C000EA020020400500203F0400208C07002058
:1051D000670500208407002080070020FFFFFBFFF9
:1051E000302B01D100F008FC0ED8192B00D16DE155
:1051F00001D201F0B0F81A2B01D001F01AFB02AB7A
:105200001A7AE24900234FE1322B01D100F010FC61
:1052100000D27EE3712B01D001F00BFB0420DC4BAC
:10522000DC4D1978C9B24A1CD2B21A70DA4A50540D
:105230001978C9B2481CC0B21870032050541978AC
:10524000C9B2481CC0B21870002050541978C9B2B5
:10525000481CC0B218702878C0B2441CE4B22C704C
:1052600050541978C9B2481CC0B21870F12318E123
:105270000625C7490C78E4B2601CC0B20870C64865
:1052800005550C78E4B2651CEDB20D700525055589
:105290000D78EDB26C1CE4B20C70002444550D780E
:1052A000EDB26E1CF6B20E7044550D78EDB26E1C68
:1052B000F6B20E70812646550D78EDB26E1CF6B230
:1052C0000E70FE2646550D78EDB26E1CF6B20E70CD
:1052D000AF214155AF49B1480B70B1490C70B1498C
:1052E0000C70016899430160AF4B1B78A34201D158
:1052F00001F09FFA2CE004218020AC4BC002196021
:10530000A6490B6803430B60A74B1B78002B1FD0EB
:10531000A74B1B88C72B1BD880214024A548836836
:105320000B438360A4488368A34383600020A34B9E
:105330001870A34B05301870A24B19701168A24B5E
:105340000B401360FA22A14B52001A6001F071FA6F
:1053500080211368C90110E0681EC0B22100FBF76C
:1053600077FC072D01D001F064FA3E2C01D001F04A
:1053700060FA8021964A090513680B43136001F017
:1053800058FA0B20824B00251978824EC9B24A1C6C
:10539000D2B21A70804A50541978C9B2481CC0B2AF
:1053A00018700A2050541978C9B2481CC0B218703D
:1053B00055541978C9B2481CC0B218703078C0B2C0
:1053C000441CE4B2347050541978C9B2481CC0B2BD
:1053D0001870842050541978C9B2481CC0B2187093
:1053E00057541978C9B2481CC0B21870555419786E
:1053F000C9B2481CC0B218703E2050541978C9B2C6
:10540000481CC0B2187073480468240E54541C78A9
:10541000E4B2611CC9B219700168090CC9B2115516
:105420001C78E4B2611CC9B219700168090AC9B2DA
:1054300011551978C9B24C1CE4B21C700368BBE268
:105440000520534B534D1978C9B24A1CD2B21A7079
:10545000514A50541978C9B2481CC0B2187004207F
:1054600050541978C9B2481CC0B21870002050546A
:105470001978C9B2481CC0B218702878C0B2441C50
:10548000E4B22C7050541978C9B2481CC0B21870DC
:10549000822050541978C9B2481CC0B2187002ABAF
:1054A0009B79535401F0C5F9D8B2824205D902ACB8
:1054B0001819407AC8540133F6E700238B540421AD
:1054C000364A02ABDF7113680B43136002ABD97924
:1054D000002900D180E000232C4AD15CD8B20029F9
:1054E00003D00133182BF8D11800294BC41D1978AB
:1054F000E4B2C9B24A1CD2B21A70274A545419787D
:10550000C9B24C1CE4B21C70841DE4B254541C7823
:10551000E4B2611CC9B21970002111551C78E4B2C3
:10552000651CEDB21D701B4DAC4661462D78EDB289
:105530006E1CF6B20E7015551C780021E4B2651C85
:10554000EDB21D70952515551C78104EE4B2651C02
:10555000EDB21D70115500211C78E4B2651CEDB24E
:105560001D7017551C78E4B2651CEDB21D70105506
:10557000CCB2844201D301F05CF91C78E4B2651C22
:10558000EDB21D70755C01311555F1E74E05002037
:10559000EA020020400500203F0400208007002090
:1055A00084070020670500201603002000E100E0CA
:1055B0007405002000400050C040005072050020DB
:1055C000B002002076050020FFFFBFDFE0020020D0
:1055D0006C050020B80200201224F84BF84E187811
:1055E000C0B2421CD2B21A70F64A14541878C0B233
:1055F000441CE4B21C70112414541878C0B2441C2A
:10560000E4B21C7011541878C0B2441CE4B21C708F
:105610003478E4B2651CEDB2357014541878C0B219
:10562000441CE4B21C70952414541878C0B2441C75
:10563000E4B21C7011541878C0B2441CE4B21C705F
:1056400011541978C9B2481CC0B2187009205054BE
:105650001978C9B2481CC0B2187042205054197849
:10566000C9B24C1CE4B21C70692454541978C9B2F4
:105670004D1CEDB21D70442555541978C9B24D1C0E
:10568000EDB21D7054541978C9B24C1CE4B21C70B0
:1056900050541978C9B2481CC0B218706F205054C9
:1056A0001978C9B24C1CE4B21C7050541978C9B2B4
:1056B000481CC0B21870732050541978C9B2481CE5
:1056C000C0B21870742050541978C9B2481CC0B2C6
:1056D0001870652050541978C9B2481CC0B21870AF
:1056E0007223DEE60720B54B00251978B44EC9B207
:1056F0004A1CD2B21A70B34A50541978C9B2481C25
:10570000C0B21870062050541978C9B2481CC0B2F3
:10571000187055541978C9B2481CC0B21870307846
:10572000C0B2441CE4B2347050541978C9B2481C59
:10573000C0B21870852050541978C9B2481CC0B244
:105740001870082050541978C9B2481CC0B218709B
:10575000575400F090FF80259B4BAD021C689B487E
:105760002C4207D01D689A4C2C401C607F23047883
:10577000234005E01C682C431C60802304782343ED
:10578000037013788E4DDBB2581CC0B21070052028
:10579000C8541378DBB2581CC0B210700420C8542F
:1057A0001378DBB2581CC0B210700020C8541378B4
:1057B000DBB2581CC0B210702878C0B2441CE4B2EE
:1057C0002C70C8541378DBB2581CC0B210708720FC
:1057D000C8541078C0B2431CDBB213707A4B1B68FC
:1057E0005B0C3B400B5401F024F80620734B002463
:1057F0001978734EC9B24A1CD2B21A70714A505409
:105800001978C9B2481CC0B21870052050541978D4
:10581000C9B2481CC0B2187054541978C9B2481C97
:10582000C0B218703078C0B2451CEDB2357050541B
:105830001978C9B2481CC0B2187086205054197823
:10584000C9B2481CC0B2187054541978C9B2481C67
:10585000C0B21870545400F0ECFF0520574B584D5F
:105860001978C9B24A1CD2B21A70564A50541978E3
:10587000C9B2481CC0B21870042050541978C9B27B
:10588000481CC0B21870002050541978C9B2481C86
:10589000C0B218702878C0B2441CE4B22C705054C6
:1058A0001978C9B2481CC0B21870882000F038FFBF
:1058B0001378434DDBB2581CC0B210700520C85499
:1058C0001378DBB2581CC0B210700420C85413788F
:1058D000DBB2581CC0B210700020C8541378DBB281
:1058E000581CC0B210702878C0B2441CE4B22C70AE
:1058F000C8541378DBB2581CC0B210708A20C85448
:105900001378DBB2581CC0B210708022CA5400F069
:1059100090FF04212F4B304D1960304B1F70304BDE
:105920001B88C72B18D840242E487C3183680B4332
:1059300083602D488368A343836000202B4B18703D
:10594000224B29707B3919701168294B0B40136069
:10595000FA22284B52001A600520184B184E19786D
:10596000C9B24A1CD2B21A70164A50541978C9B238
:10597000481CC0B21870042050541978C9B2481C91
:10598000C0B21870002050541978C9B2481CC0B277
:1059900018703078C0B2441CE4B234705054197896
:1059A000C9B2481CC0B21870B02050541978C9B29E
:1059B000481CC0B218702B78DBB272E5EA020020F6
:1059C000400500203F04002080070020B002002096
:1059D000FFFFFDFF00E100E07605002066050020E6
:1059E0007405002000400050C040005072050020A7
:1059F000FFFFBFDFE00200208020CA498B6883439D
:105A00008B60C94940388B6803438B600023C749CA
:105A10000B70C7490878052801D1023000E0062044
:105A20000870C4490B708121136889050B4313600A
:105A30000F20C14BC14D1978C9B24A1CD2B21A709D
:105A4000BF4A50541978C9B2481CC0B2187004201B
:105A500050541878C0B2411CC9B2197000211154B9
:105A60001878C0B2441CE4B21C702C78E4B2661CF6
:105A7000F6B22E7014541878C0B2441CE4B21C70F4
:105A8000B02414541878C0B2441CE4B21C70A94C61
:105A9000A4462478E4B214541878C0B2441CE4B28A
:105AA0001C70092414541878C0B2441CE4B21C7051
:105AB00011541878C0B2441CE4B21C702C78E4B2C3
:105AC000661CF6B22E7014541878C0B2441CE4B2AE
:105AD0001C70B22414541878C0B2441CE4B21C7078
:105AE00017541878C0B2441CE4B21C706446247881
:105AF00064B28C4204DA93494C780A216143C9B2FA
:105B000011541978C9B2481CC0B218700020505402
:105B10001978C9B24C1CE4B21C7050541978C9B23F
:105B20004C1CE4B21C70022454541978C9B24C1CA9
:105B3000E4B21C70505400F07CFE834B1A687E4B1C
:105B4000520331D5052019787C4DC9B24A1CD2B216
:105B50001A707B4A50541978C9B2481CC0B21870E8
:105B6000042050541978C9B2481CC0B218700020E3
:105B700050541978C9B2481CC0B218702878C0B205
:105B8000441CE4B22C7050541978C9B2481CC0B2FD
:105B90001870B02050541978C9B2481CC0B218709F
:105BA00064480078C0B25054052019780025C9B265
:105BB0004A1CD2B21A70624A604E50541978C9B267
:105BC000481CC0B21870042050541978C9B2481C3F
:105BD000C0B2187055541978C9B2481CC0B21870B8
:105BE0003078C0B2441CE4B2347050541978C9B251
:105BF000481CC0B21870922050541978C9B2481C81
:105C0000C0B2187012235354504B1D7000F011FE97
:105C100002AB9B794D4A152B37D013D8102B2CD0C3
:105C200007D80C2B3FD00F2B25D00B2B3DD10E23AB
:105C30003AE0122B25D022D3132B24D0142B34D1AD
:105C4000052331E01A2B26D008D8172B21D01ED3DC
:105C5000182B26D0192B28D10D2325E0FC2B1ED084
:105C600003D81C2B21D110231EE0FD2B15D0FE2BB9
:105C70001BD1112318E0002316E0177015E0022352
:105C800012E0032310E004230EE006230CE00723B8
:105C90000AE0082308E0092306E00A2304E00B23B6
:105CA00002E00C2300E00F23137006200525224B91
:105CB000224E1978C9B24A1CD2B21A70204A5054E6
:105CC0001978C9B2481CC0B2187055541978C9B2B5
:105CD000481CC0B21870002050541978C9B2481C32
:105CE000C0B218703078C0B2441CE4B23470174CA3
:105CF00050542178112900D9AFE1080000F0FEFFCF
:105D0000280036004C00610077008D00A300B10030
:105D1000DE00F4000B012001350143015B01690144
:105D20007F01960100400050C040005066050020F1
:105D3000B002002076050020EA0200204005002085
:105D40003F040020EB0200208007002068020020B2
:105D50001878C0B2451CEDB21D7090251554187806
:105D6000C0B2451CEDB21D700F2522E01878C0B2FC
:105D7000451CEDB21D70902515541878C0B2451C15
:105D8000EDB21D70102515541878C0B2451CEDB247
:105D90001D70E54B5B7847E11878C0B2451CEDB249
:105DA0001D70902515541878C0B2451CEDB21D70B9
:105DB000112515541878C0B2451CEDB21D7017544A
:105DC00060E11878C0B2451CEDB21D7090251554E5
:105DD0001878C0B2451CEDB21D7012251554187804
:105DE000C0B2451CEDB21D70CF4B5B79E1E0187875
:105DF000C0B2451CEDB21D70902515541878C0B284
:105E0000451CEDB21D70132515541878C0B2451C01
:105E1000EDB21D70C44B9B7806E11878C0B2451CEA
:105E2000EDB21D70902515541878C0B2451CEDB226
:105E30001D70142515541878C0B2451CEDB21D70A4
:105E4000B94BDB78F0E01878C0B2451CEDB21D709C
:105E5000902515541878C0B2451CEDB21D7015255B
:105E6000A7E71878C0B2451CEDB21D7090251554F7
:105E70001878C0B2451CEDB21D7016251554AA48FD
:105E80000079C0B203280BD0042810D0022800D01B
:105E9000F8E01878C0B2451CEDB21D708B23F0E01D
:105EA0001878C0B2451CEDB21D709B23E9E018784C
:105EB000C0B2451CEDB21D70AA23E2E01878C0B252
:105EC000451CEDB21D70902515541878C0B2451CC4
:105ED000EDB21D70172515541878C0B2451CEDB2EF
:105EE0001D70914B9B799FE01878C0B2451CEDB2B4
:105EF0001D70902515541878C0B2451CEDB21D7068
:105F00001A2515541878C0B2451CEDB21D70864B89
:105F10005B795B084DE01878C0B2451CEDB21D708E
:105F2000902515541878C0B2451CEDB21D70FD25A2
:105F300015541878C0B2451CEDB21D700823A0E0BE
:105F40001878C0B2451CEDB21D7090251554187814
:105F5000C0B2451CEDB21D70FC2515541878C0B2B6
:105F6000451CEDB21D7018238BE01878C0B2451C9B
:105F7000EDB21D70902515541878C0B2451CEDB2D5
:105F80001D70182515E71878C0B2451CEDB21D70BC
:105F9000902515541878C0B2451CEDB21D70192516
:105FA00015541878C0B2451CEDB21D705E4B5B797C
:105FB0009B093B4065E01878C0B2451CEDB21D70EE
:105FC000902515541878C0B2451CEDB21D700B25F4
:105FD00039E01878C0B2451CEDB21D7090251554FB
:105FE0001878C0B2451CEDB21D700C2515541878F8
:105FF000C0B2451CEDB21D704B4BDB7C14E0187831
:10600000C0B2451CEDB21D70902515541878C0B271
:10601000451CEDB21D701C2515541878C0B2451CE6
:10602000EDB21D70404B9B7CDBB22AE01878C0B209
:10603000451CEDB21D70902515541878C0B2451C52
:10604000EDB21D70FE2515541878C0B2451CEDB296
:106050001D70354B5B79DB0913E018780438155453
:1060600004251878033815541878C0B2451CEDB2D1
:106070001D70912515541878C0B2451CEDB21D70E5
:10608000FF23135401312170D3E3284C284D23788A
:106090000020DBB25A1CD2B222700622EA542378C6
:1060A000244EDBB25A1CD2B222700522EA54237865
:1060B000DBB25A1CD2B22270E8542378DBB25A1CED
:1060C000D2B222703278D2B2511CC9B23170EA54C5
:1060D0002378DBB25A1CD2B222709022EA54227882
:1060E000D2B2531CDBB2237002AB9B79AB54142B9E
:1060F0005CD035D8102B00D1AEE01DD80B2B00D1D1
:10610000E3E00C2B00D01EE123781220DBB25A1CF6
:10611000D2B2227002AAD4792100EC54FAF798FD89
:10612000014BDC7485E3C046EB020020EA0200204C
:106130003F04002040050020122B24D0132B00D058
:1061400001E123780120DBB25A1CD2B2227002AAEC
:10615000D4792100EC54FAF77BFDDA4B9C7068E3AC
:10616000192B00D198E004D8162B35D0172B5DD011
:10617000E9E01C2B00D1C1E0FE2B00D1CDE01A2BB1
:1061800000D0E0E076E0CF4E02AA7379D079227891
:10619000DBB2D2B2511CC9B22170002802D0AF5478
:1061A0003B4301E0A854BB431C00A1E002ABDB79F8
:1061B000FA2B02D9FA2302AAD37123780220DBB288
:1061C0005A1CD2B2227002AAD4792100EC54FAF7F8
:1061D0003FFDBC4BDC702CE302ABDB79B94EAA2B44
:1061E00008D9AA2302AA04210320D371FAF730FDAB
:1061F000042312E09A2B08D88B2302AA0221032041
:10620000D371FAF725FD022307E003219B2302AA9D
:106210000800D371FAF71CFD032333712378DBB236
:106220005A1CD2B2227002AAD27992E002ABDB7978
:10623000632B02D8002302AAD37123780520DBB296
:106240005A1CD2B2227002AAD4792100EC54FAF777
:10625000FFFC9C4B9C71ECE22378DBB25A1CD2B25F
:10626000227002AAD4792100EC54FAF7F1FC954B84
:106270005C70DEE2934E02AA7379D0792278DBB2A9
:10628000D2B2511CC9B22170002802D0AF540224EE
:1062900029E0A854022216E08A4E02AA7379D27924
:1062A000DBB2002A07D02278D2B2511CC9B22170C9
:1062B000AF54402417E02278D2B2511CC9B22170E9
:1062C0000021A954402293436EE77E4E02AA7379BF
:1062D000D0792278DBB2D2B2511CC9B22170002829
:1062E00003D08024AF541C4302E07F24A8541C40F8
:1062F00021000420FAF7ACFC74719AE22378112093
:10630000DBB25A1CD2B2227002AAD4792100EC541A
:10631000FAF79EFC6B4B9C748BE222780420D2B27D
:10632000531CDBB2237002ABDB79AB547F22654D8B
:106330006C7914405A1E9341DB011C432100FAF78B
:1063400087FC6C7175E22378DBB25A1CD2B22270E2
:106350000022EA546DE202AB9A795B4B1A7002AAF2
:10636000D2795A7002AA127A9A7002AA527ADA7014
:106370005FE202AB9A79092A05D802A81318DB79E3
:106380009C46092B08D90A68504B13400B600A68D9
:106390004F4B13400B60D1E34E4B1C78E4B2611CB1
:1063A000C9B2197061465018C0B24B49851DEDB293
:1063B0000D551C780530E4B2651CEDB2C0B21D70FD
:1063C00008551C78E4B2601CC0B218700020085553
:1063D0001C784248E4B2651CEDB21D703F4D2D782B
:1063E000EDB26E1CF6B206700D551C780020E4B2BA
:1063F000651CEDB21D7093250D551C780090E4B21C
:10640000651CEDB21D700A551C0068460578AA424D
:106410000ED9257802A8EDB26E1CF6B22670009E49
:106420003618F6792C484655009801300090ECE774
:106430001878C0B2451CEDB21D7063460B540023A2
:10644000D9B28C450CD9217802ADC9B2481CC0B272
:10645000207098184019007A1F4D01336854EFE7F7
:1064600002ABDD790A210023303DEDB20133D8B211
:10647000824207D902AC4D431819C07930382D1823
:10648000EDB2F3E702A953180A2000211C7A303C30
:10649000E4B20131CBB29C4501D8FEF75DFF8B1809
:1064A00002AE44439B191B7A303BE418E4B2F0E798
:1064B00002AB9979092913D91168044B0B40136079
:1064C00038E3C046EB020020E6020020FFFFFFFD9C
:1064D000FFFFFFFBEA0200203F04002040050020F0
:1064E00000220A2002ABDB79303BDBB200930132A1
:1064F000D3B299420AD902AC1319DC79009D23006A
:106500004543303BEB18DBB20093F0E7009B072BD1
:1065100002D10822E74BDA710800E74C09302278F3
:10652000C0B2D2B2531CDBB22370E44B9854227831
:10653000D2B2501CC0B2207008000830C0B29854CB
:106540002078C0B2421CD2B2227000221A542078A5
:10655000C0B2451CEDB22570D94DAC4662462D78CF
:106560009C46EDB26E1CF6B216701D5420780022C7
:10657000C0B2451CEDB22570932526001D5420782D
:10658000C0B2451CEDB225701954D0B288420BD26E
:10659000307802ABC0B2451CEDB23570D5186346F9
:1065A000ED7901321D54F0E72378C44DDBB25A1C5B
:1065B000D2B222700322EA542678009AF6B2731CF3
:1065C000DBB22370BB4B6421985CC0B200F0A0FB2F
:1065D0003030009AB74BC0B2A855985C6421C0B265
:1065E00000F01CFC2678CBB2F6B20093731CDBB231
:1065F00023700A21009800F08BFB3030C0B2A85500
:1066000026780A21F6B2731CDBB22370009800F0E2
:1066100005FC3031C9B2A9550BE105201168A94B21
:1066200000250B401360A44BA54E1978C9B24A1C33
:10663000D2B21A70A14A50541978C9B2481CC0B2DB
:106640001870042050541978C9B2481CC0B2187090
:1066500055541978C9B2481CC0B218703078C0B20D
:10666000441CE4B2347050541978C9B2481CC0B20A
:106670001870942050541978C9B2481CC0B21870D0
:106680005554D6E0904802A90368497A1B0E9942F6
:1066900000D0CEE002AB9C7AFF230168090C1940C0
:1066A0008C4200D0C5E0016802ACE47A090A1940C6
:1066B0008C4200D0BDE002A90068097B03409942EA
:1066C00000D0B6E080210520136889040B431360D5
:1066D000794B7B4D1978C9B24A1CD2B21A70774AED
:1066E00050541978C9B2481CC0B2187004205054D4
:1066F0001978C9B2481CC0B21870002050541978DB
:10670000C9B2481CC0B218702878C0B2441CE4B2A8
:106710002C7050541978C9B2481CC0B2187094201B
:1067200050541978C9B2481CC0B21870575480E050
:1067300002AB9B79002B7CD102AB5B7A3E2B78D1EC
:10674000614902AA0B68927A1B0E9A4271D102AB80
:10675000D87AFF230A68120C1A40904269D10A685D
:1067600002A8007B120A1A40904262D102AA09686C
:10677000527B0B409A425CD1FAF75CFAFAF742FA84
:10678000F8204002FAF714FA2378504A504C1B02C2
:106790001343236021684F48FAF7B2F903214E4AA8
:1067A00013680B432360236813604C4A4C4B1A60F8
:1067B000FEE780204B498B6883438B604A49403811
:1067C0008B6803438B60FA21484B890019800021B4
:1067D0008120474B80051970136803431360454AB5
:1067E000454B1068034090201360444A936803436C
:1067F00093608022424B9201DA67424B424A197001
:10680000424BFF311A60424A11701A68002AFCD1CB
:106810002B4B1A70FAF70EFA03212F4A13680B4319
:1068200013602E4A2E4B1A60A022D20593683B4378
:10683000936002AB9B78002B00D063E102AA12792F
:10684000092A00D1F9E00AD8032A00D12CE1042A50
:1068500000D057E1274A284B11680B4051E1302AFC
:1068600000D19BE0312A00D04CE10421294A204C80
:106870001160294A1770294A1188294AC72957D80F
:1068800080204026174DA9680143A960164DA968CC
:10689000B143A96023490B700521234B1970207067
:1068A0001168224B0B401360FA22184B52001A60F9
:1068B00043E0C046EB020020EA0200203F04002033
:1068C00040050020FFFFFFFDB80200203E00FFFF53
:1068D000D00200201CF0010000C000500400FA05A6
:1068E0000CED00E000400050C0400050E4020020E9
:1068F0007605002080070020FFFFFBFF804000504E
:1069000004E100E094070020DC050000E002002024
:106910003D04002000E100E0660500207405002031
:106920006C05002072050020B0020020FFFFBFDFD1
:1069300080211368C9010B4313600520804B814EF1
:106940001978C9B24A1CD2B21A707F4A50541978C9
:10695000C9B2481CC0B21870042050541978C9B28A
:10696000481CC0B21870002050541978C9B2481C95
:10697000C0B218703078C0B2451CEDB235705054BA
:106980001978C9B2481CC0B21870B0205054197898
:10699000C9B2481CC0B2187023784BE080206B4904
:1069A0008A6882438A606A4940388A6802438A60FA
:1069B000684A1370684B1A78052A01D1023200E048
:1069C0000622002081210524644D1A70644A287033
:1069D000136889050B431360594B5A4E1978C9B295
:1069E0004A1CD2B21A70584A54541978C9B24C1C75
:1069F000E4B21C70042454541978C9B24C1CE4B29B
:106A00001C7050541978C9B2481CC0B21870307844
:106A1000C0B2441CE4B2347050541978C9B2481C56
:106A2000C0B21870B02050541978C9B2481CC0B216
:106A300018702B78DBB2535464E0802043498A6895
:106A400082438A60424940388A6802438A60FA2158
:106A50008120444A89001180404A414913700A68E4
:106A6000800502430A6080213F4A8901D167FF21E6
:106A70003E4A13703E4A3F4B1A603F4A11701A68F3
:106A8000002AFCD12F4B1A70FAF7D4F803213B4AA5
:106A900013680B4313603A4A3A4B1A60A022D2059E
:106AA00093683B4393602DE080203749C0020A6819
:106AB00002430A60354A1178294A00291DD0344919
:106AC0000988C72919D880204025204CA168014396
:106AD000A1601F4CA168A943A1602E490B7005213C
:106AE0001D4B19701D4B187011682B4B0B40136018
:106AF000FA22204B52001A6004E080211368C90179
:106B00000B43136002AB1A785B7801339A4210DDB5
:106B1000DBB2D21A02A90A70002201320198D1B266
:106B2000884201D8FEF75DFA02A81918895C8154E1
:106B3000F3E70B4A1168194B0B40136013B0F0BD1B
:106B4000EA020020400500203F04002000400050E1
:106B5000C040005066050020B002002076050020ED
:106B60006C050020E402002004E100E0940700200E
:106B7000DC050000E00200203D04002000C00050C1
:106B80000400FA050CED00E0800700201603002049
:106B90007405002072050020FFFFBFDFFFFFFFFB31
:106BA000F7B508AC247880250194A024E405E768B3
:106BB0006D052F43E760E668204F3740E760204CC3
:106BC00003273B409F0063690C26B3433B4363614B
:106BD000019F1C4B3E04A7693B403343A361A3685C
:106BE0001D43194BA5601C6A01252C431C621C6ABD
:106BF000002802D11548204002E08020C000204338
:106C000018620C20002902D1196A814305E001298C
:106C100005D1196A814304200143196208E0022961
:106C200003D1196A81430820F6E7196A08431862FC
:106C3000596AFF2081430A435A62F7BDFFFFFFEF05
:106C400000020050FFFF00FF00000E40FFFBFFFFAF
:106C500010B5194C236BDA070CD5184A1368002BB2
:106C600001D050689847164B07211A688A430121C2
:106C70000A431A60236B9A070CD5104A1369002B3C
:106C800001D0906898470E4B07211A688A43022169
:106C90000A431A60236B5A070CD5084A5369002B24
:106CA00001D0D0689847064B07211A688A4304210F
:106CB0000A431A6010BDC04600000E408C0200203E
:106CC00030000E40064B07211A688A4301210A430F
:106CD0001A60044B8022196A12010A431A62704733
:106CE00030000E4000000E4002B4714649084900D1
:106CF000095C49008E4402BC7047C04603B471462B
:106D0000490840004900095A49008E4403BC7047B5
:106D1000002243088B4274D303098B425FD3030ADA
:106D20008B4244D3030B8B4228D3030C8B420DD3ED
:106D3000FF22090212BA030C8B4202D3121209027B
:106D400065D0030B8B4219D300E0090AC30B8B42B9
:106D500001D3CB03C01A5241830B8B4201D38B0367
:106D6000C01A5241430B8B4201D34B03C01A52410C
:106D7000030B8B4201D30B03C01A5241C30A8B424F
:106D800001D3CB02C01A5241830A8B4201D38B023A
:106D9000C01A5241430A8B4201D34B02C01A5241DE
:106DA000030A8B4201D30B02C01A5241CDD2C30950
:106DB0008B4201D3CB01C01A524183098B4201D3CC
:106DC0008B01C01A524143098B4201D34B01C01AB7
:106DD000524103098B4201D30B01C01A5241C3082F
:106DE0008B4201D3CB00C01A524183088B4201D39E
:106DF0008B00C01A524143088B4201D34B00C01A8A
:106E00005241411A00D20146524110467047FFE7F5
:106E100001B5002000F0F0F802BDC0460029F7D00F
:106E200076E7704703460B437FD4002243088B422A
:106E300074D303098B425FD3030A8B4244D3030B01
:106E40008B4228D3030C8B420DD3FF22090212BAC6
:106E5000030C8B4202D31212090265D0030B8B4242
:106E600019D300E0090AC30B8B4201D3CB03C01A2C
:106E70005241830B8B4201D38B03C01A5241430B07
:106E80008B4201D34B03C01A5241030B8B4201D3F7
:106E90000B03C01A5241C30A8B4201D3CB02C01A62
:106EA0005241830A8B4201D38B02C01A5241430ADA
:106EB0008B4201D34B02C01A5241030A8B4201D3C9
:106EC0000B02C01A5241CDD2C3098B4201D3CB0170
:106ED000C01A524183098B4201D38B01C01A52411F
:106EE00043098B4201D34B01C01A524103098B4223
:106EF00001D30B01C01A5241C3088B4201D3CB000E
:106F0000C01A524183088B4201D38B00C01A5241F0
:106F100043088B4201D34B00C01A5241411A00D2A0
:106F200001465241104670475DE0CA0F00D0494209
:106F3000031000D34042534000229C4603098B4279
:106F40002DD3030A8B4212D3FC22890112BA030A01
:106F50008B420CD3890192118B4208D38901921183
:106F60008B4204D389013AD0921100E08909C30908
:106F70008B4201D3CB01C01A524183098B4201D30A
:106F80008B01C01A524143098B4201D34B01C01AF5
:106F9000524103098B4201D30B01C01A5241C3086D
:106FA0008B4201D3CB00C01A524183088B4201D3DC
:106FB0008B00C01A5241D9D243088B4201D34B00F7
:106FC000C01A5241411A00D20146634652415B1039
:106FD000104601D34042002B00D54942704763461A
:106FE0005B1000D3404201B5002000F005F802BD5F
:106FF0000029F8D016E770477047C046000000002F
:1070000020000000000010002000100030353A3F42
:1070100044494E54585C61666B7075A512646403F4
:1070200081C8083E041EFFFFFFFFFFFFFF0530FF82
:10703000020408100100000002000000020000002D
:047040000400000048
:10704400FF404040404040403340404034403536AB
:1070540040404040404040403A4040403B403C3744
:10706400404040403F403D3840403E3940FB404076
:107074004040404040404040244040402340222182
:10708400404040401F401E2040401D1C401B4040CB
:10709400404040401940181A4040171640154040DF
:1070A400404025144013404040324040404040405E
:1070B4004040404040404040FE4040400E400D0CA7
:1070C400404040400A40090B404008074006404009
:1070D400404040400440030540400201400040401D
:1070E40040400F104011404040124040404040405A
:1070F40040404040FD402B3040402A2F403140402A
:107104004040292E402D4040402C404040404040CB
:107114004040FA28402740404026404040404040FC
:1071240040FC0000001BB70000000000008051017B
:10713400102700000080510100805101160000005A
:00000001FF
